:020000040800F2
:100000002052042459030008736100087F2D000862
:100010006503000841080008B576000800000000EC
:10002000000000000000000000000000EB6D000870
:10003000590A000800000000756100089D6E000864
:1000400073030008730300087303000873030008B8
:1000500073030008730300087303000873030008A8
:100060007303000873030008730300087303000898
:100070007303000873030008730300087303000888
:100080007303000873030008730300087303000878
:100090007303000873030008730300087303000868
:1000A0007303000873030008730300087303000858
:1000B0007303000873030008730300087303000848
:1000C0007303000873030008730300087303000838
:1000D00073030008717600087303000873030008B7
:1000E0007303000873030008000000007303000896
:1000F0007303000873030008730300087303000808
:1001000073030008730300087303000873030008F7
:1001100073030008730300087303000873030008E7
:1001200073030008730300087303000873030008D7
:1001300073030008730300087303000873030008C7
:1001400000000000000000000000000000000000AF
:1001500073030008730300087303000873030008A7
:100160007303000873030008730300087303000897
:100170007303000873030008730300087303000887
:100180007303000873030008730300087303000877
:100190007303000873030008730300087303000867
:1001A0007303000873030008730300087303000857
:1001B0007303000873030008730300087303000847
:1001C0007303000873030008730300087303000837
:1001D0007303000873030008730300087303000827
:1001E0007303000873030008730300087303000817
:1001F0007303000873030008730300087303000807
:1002000073030008730300087303000873030008F6
:1002100073030008730300087303000873030008E6
:100220007303000873030008730300080000000054
:100230007303000873030008000000007303000844
:1002400073030008730300087303000873030008B6
:1002500073030008730300087303000873030008A6
:100260007303000873030008730300087303000896
:100270007303000873030008730300080000000004
:100280007303000800000000730300080000000072
:10029000000000007303000800F002F800F044F8CA
:1002A0000AA090E8000C82448344AAF10107DA45D1
:1002B00001D100F039F8AFF2090EBAE80F0013F0DF
:1002C000010F18BFFB1A43F001031847E8C00000F4
:1002D00008C10000103A24BF78C878C1FAD8520784
:1002E00024BF30C830C144BF04680C6070470000B0
:1002F0000023002400250026103A28BF78C1FBD82F
:10030000520728BF30C148BF0B607047642900F016
:10031000FB80782900F03481002070471FB507F07A
:1003200057FC1FBD10B510BD00F058FA1146FFF77D
:10033000F5FF07F00DFA00F076FA03B4FFF7F2FFCD
:1003400003BC07F0C8F9000030BF72B6704762B650
:10035000704780F30888704709488047094800477C
:10036000FEE7FEE7FEE7FEE7FEE7FEE7FEE7FEE765
:10037000FEE7FEE704480549054A064B70470000C2
:10038000A16E00089902000820460424205204248B
:10039000204804242048042453EA020C00F0698019
:1003A0002DE9F04B4FF00006002B1FBFB3FA83F589
:1003B00003FA05F424FA05F65E4012BF1643B2FABA
:1003C00082F502FA05F4C5F120051EBF22FA05FCEC
:1003D00044EA0C04203556EA044C4FEA144418BF92
:1003E000641C4FF000084FF00009904271EB030CC1
:1003F00039D3002919BFB1FA81F701FA07F6B0FA2B
:1004000080F700FA07F6C7F120071EBF20FA07FCA5
:1004100046EA0C062037B6FBF4FCA7EB0507103FB5
:1004200007F01F0BCBF120060CFA0BFB2CFA06F69B
:1004300044BFB3460026202FA4BF5E464FF0000BFA
:100440005BEA060C08BF4FF0010B19EB0B09ABFB85
:10045000027C48EB0608C01B06FB02CC0BFB03CC5E
:1004600071EB0C01C1E70B46024641464846BDE828
:10047000F08B13B54FF000004FF00001AFF3008098
:10048000BDE81C40704700000FB4044910B503AA32
:10049000029800F075F910BC5DF814FB1000002400
:1004A0002DE9F0410E460446002020622046E16816
:1004B000884730B3252805D0D4E901219047206A28
:1004C000401CF2E7E168204600278847050018D065
:1004D000A5F14100192802D820354FF400673246B3
:1004E000294620462760FFF711FF40B1012804D0BC
:1004F000F61D26F007060836D8E7361DD6E728464B
:10050000DAE7206ABDE8F0812DE9F04106460024D3
:1005100010687529314616A510D0AFF30080002869
:1005200002DA404213A507E031688A0701D512A517
:1005300002E0490704D511A5012401E0AFF30080D2
:1005400000210A2206F1240709E0B0FBF2FCB0FB0F
:10055000F2F302FB1C00303078541846491C002886
:10056000F3D123462A463046BDE8F04100F0AEB84C
:10057000000000002D0000002B0000002000000003
:1005800070B504460D4621461068AFF300802188FF
:10059000090502D50F4A7A4402E00E4A7A440E3227
:1005A000002104F1240305E000F00F060009965D28
:1005B0005E54491C0028F7D120780023000704D599
:1005C000702D02D009B1022311322046BDE87040DF
:1005D00000F07CB8F2BD0000032A40F2308010F039
:1005E000030C00F0158011F8013BBCF1020F6244CE
:1005F00098BF11F801CB00F8013B38BF11F8013B5F
:10060000A2F1040298BF00F801CB38BF00F8013B0B
:1006100011F0030300F02580083AC0F0088051F87B
:10062000043B083A51F804CBA0E80810F5E7121D86
:100630005CBF51F8043B40F8043BAFF30080D207A5
:1006400024BF11F8013B11F801CB48BF11F8012B71
:1006500024BF00F8013B00F801CB48BF00F8012B94
:10066000704710B5203AC0F00B80B1E81850203A1E
:10067000A0E81850B1E81850A0E81850BFF4F5AF42
:100680005FEA027C24BFB1E81850A0E8185044BFCC
:1006900018C918C0BDE810405FEA827C24BF51F839
:1006A000043B40F8043B08BF7047D20728BF31F82D
:1006B000023B48BF11F8012B28BF20F8023B48BF7E
:1006C00000F8012B70477047704770472DE9F047DD
:1006D0000D4699469246044600F1240801688806B2
:1006E00004D5E06921F01001216000E00120A8425A
:1006F00001DD471B00E00027A1697A1902EB090020
:10070000081AA0612078C00602D42046AFF300800A
:10071000002608E0D4E901211AF806009047206A73
:10072000401C761C20624E45F4DB2078C0060AD5BA
:100730002046AFF3008006E0D4E901213020904745
:10074000206A401C2062381EA7F10107F4DC07E094
:10075000D4E9012118F805009047206A401C206266
:10076000281EA5F10105F3DC2046AFF300802078B8
:10077000000602D50220BDE8F0870120FBE700005B
:10078000074B70B50D467B4400F011F8044628462F
:1007900000F020F810B14FF0FF3070BD204670BD62
:1007A000B36F000001694A1C02610878704700B508
:1007B0008FB0CDE901310021059105497944CDE99A
:1007C000031011466846FFF76BFE0FB000BD000036
:1007D000E5FFFFFF007B00F080007047754600F0EA
:1007E0002BF8AE4605006946534620F007008546C3
:1007F00018B020B5FFF7BEFDBDE820404FF0000661
:100800004FF000074FF000084FF0000B21F00701F8
:10081000AC46ACE8C009ACE8C009ACE8C009ACE83B
:10082000C0098D46704710B50446AFF300802046DE
:10083000BDE81040FFF781BD00487047C045042463
:10084000FEE70000F0B5BFF34F8FBFF36F8F1D4978
:1008500000200860BFF34F8FBFF36F8F1A4C2168E1
:1008600041F400312160BFF34F8FBFF36F8F164902
:1008700070310860BFF34F8F081F006843F6FF75A3
:10088000104E1036C0F34E31C0F3C90305EA4112D1
:10089000184642EA80773760401EFAD2491EF5D2E8
:1008A000BFF34F8F206840F480302060BFF34F8F3C
:1008B000BFF36F8F03484C30016841F004010160C1
:1008C000F0BD000050EF00E014ED00E0084A002009
:1008D0004FF4803102E0536B1B0602D4491EFAD25A
:1008E00000E011B103499163704703207047000095
:1008F00000700052FF0FE01F0E4A10B5516B11F04F
:10090000450FFBD00C4B4C0704D504209063936338
:10091000032010BDC90702D00120906310BD1169EA
:10092000814201D0102010BD9363506900F008008F
:1009300010BD000000700052FF0FE01F10B50F4CFB
:1009400000204FF480320BE0616B11F0450F07D0AF
:100950000AB14A0707D5A16B032041F004010AE060
:10096000521EF1D2F5E7C90704D0A16B012041F076
:100970000101A1630249A16310BD00000070005293
:10098000FF0FE01F0849486B10F0450FFBD04007F0
:1009900005D5886B40F00400886303207047034846
:1009A000886300207047000000700052FF0FE01FB6
:1009B00030B5174B054600205A6B12F0450FFBD09F
:1009C000540705D5986B40F004009863032030BDB0
:1009D000D20705D0986B40F001009863012030BD2C
:1009E0001A69AA420ED10B4A9A635A6912F4604FEF
:1009F00003D0910404D5132030BD120C0A8030BD01
:100A0000510401D5102030BD1104FCD50F2030BD9C
:100A100000700052FF0FE01F10B50E4C00204FF485
:100A200080320BE0616B11F0450F07D00AB14A0725
:100A300007D5A16B032041F0040108E0521EF1D25A
:100A4000F5E7490604D5A16B002041F04001A16300
:100A500010BD0000007000527047000070B5B3F583
:100A6000804F05D06FF0704140F82210002070BD1B
:100A700050F82230084C2340D1E900458E8944EAE1
:100A800005148D6889692D0245EA06452C430C43FF
:100A90001C4340F82240E9E70000F0CFF0B50C68B5
:100AA00050F824501A4A1540D1E90123D1E90367CF
:100AB0001A433E4332434E6932438E693243CE6914
:100AC00032430E6A32434E6A32438E6A3243CE6AF2
:100AD00032430E6B32438E6B32434E6B32432A43AA
:100AE000082B01D142F0400240F824200A6BB2F5F5
:100AF000801F05D10A684AB1026842F48012026080
:100B00000A681AB10268496B0A4302600020F0BD0E
:100B10008004C0FF00EB8202F0B553688E8903F0B9
:100B20004044D1E9003543EA05138D682D0245EABA
:100B300006450E8A2B430D4D05EB065633430E7DBD
:100B40006F0107EB066633438E69334323435360DB
:100B50000268D20207D54268098A22F4700205EBC6
:100B60000151114341600020F0BD00000000F0FF82
:100B700030B5D1E901230D681A43D1E90334234389
:100B80001A434B691A438B691A43D1E90734496AFE
:100B9000012D056807D01A4322430A436FF30E055F
:100BA0002A4302600AE025F4F845234329430B4316
:100BB000416803606FF30E010A434260002030BDBC
:100BC000426942EA410141610020704718B5D1E90C
:100BD00000236FF01F041A438B68C96804EB4313AA
:100BE00043EA41210A4300920261002018BD00003F
:100BF000F0B5D1E900346FF00F055B1E2E0105EB57
:100C0000041423438C682F034FEA054C0D8A06EB2E
:100C100004248E8A2343CC68097E4FF07F4E012A3C
:100C200007EB05450CEB06560EEB01610CD0826814
:100C30003F1107EB043423432B4333430B4302F0B0
:100C40007042134383600FE08768084A174022030D
:100C5000C468A2F5805232433A4382602B430B436F
:100C600004F070442343C3600020F0BDFF0F0FFF6A
:100C7000F0B500240E460822074601212546102023
:100C800005F062FC1020FFF737FE00282ED13A0451
:100C90000121372005F058FC3720FFF72DFE0028F2
:100CA00024D1012303220821401E05F059FC002213
:100CB0000121332005F048FC3320FFF71DFE0028FA
:100CC00014D1174940F22A524B6B134206D14B6B99
:100CD0001B03F9D4D1F88040D1F880504A6B120739
:100CE00005D5886B40F0080088630420F0BD4A6B8E
:100CF000920705D5886B40F0020088630220F0BDA2
:100D00004A6B920605D5886B40F020008863062068
:100D1000F0BD044A8A6321BA716029BA3160F0BD1E
:100D200000700052FF0FE01F10B528B190F8351089
:100D3000022903D080214165012010BD1D4A4FF4D6
:100D4000956301688C189C4207D8042280F83520EE
:100D5000086820F00100086029E00C6824F00E0407
:100D60000C6001680A440A6822F001020A60016E00
:100D70000A6822F480720A6090F85C30012202FA5C
:100D800003F10D4B1960D0E919134B60C16E31B1FD
:100D90000B6823F480730B60D0E91C134B600021B7
:100DA00080F8341080F83520016D01B188470020AB
:100DB00010BD0000F0FFFDBF045402580248016856
:100DC00041F0010101607047200400582DE9F84FFF
:100DD0006C4C00224FF0B04A4FF0010B4FF0030E65
:100DE0004FF00F090B680BFA02F73B40BB4270D182
:100DF0004D68022D01D0122D12D1D50800EB850CC3
:100E0000DCF820605507ED0E09FA05F826EA080619
:100E1000D1F8108008FA05F848EA0608CCF82080D6
:100E2000D0F80080560091F804C00EFA06F50CF0D8
:100E3000030C28EA05080CFA06FC4CEA080CC0F87A
:100E400000C0D1F804C0BCF1010F08D0BCF1020F02
:100E500005D0BCF1110F02D0BCF1120F16D1D0F8A1
:100E600008C0D1F80C802CEA050C08FA06F848EA0C
:100E70000C08C0F80880D0F804C02CEA070C0F79E1
:100E8000C7F30017974047EA0C074760C768AF43AE
:100E90008D68B5403D43C5604D68ED006BD53A4D5A
:100EA0002E6846F002062E602D6822F0030606F139
:100EB000B04605F002050095D6F808C495072F0F37
:100EC00009FA07F52CEA050C304DA84202D100259D
:100ED0002EE050E02E4DA84201D1012528E02D4DF5
:100EE000A84201D1022523E02B4DA84201D10325C0
:100EF0001EE02A4DA84201D1042519E0284DA84240
:100F000001D1052514E0274DA84201D106250FE0A7
:100F1000254DA84201D107250AE0244DA84201D160
:100F2000082505E0224DA84201D1092500E00A2547
:100F3000BD4045EA0C05C6F8085425684E689D4337
:100F4000F60300D51D43256065684E689D43B603D2
:100F500000D51D436560DAF8005056464F689D4342
:100F6000FF0200D51D43356075684F689D43BF0281
:100F700000D51D437560521C102AFFF433AFBDE845
:100F8000F88F000080000058F44402580000025816
:100F90000004025800080258000C025800100258C1
:100FA0000014025800180258001C02580020025871
:100FB000002402580069084000D0012070474269AF
:100FC0004A40426170470AB10183704741837047CC
:100FD00001488068704700001400002402488168BE
:100FE000027811448160704714000024032010B57A
:100FF00000F0FCF90F2000F007F808B1012010BD47
:1010000000F0C6F9002010BD70B50D4D04464FF438
:101010007A712878B1FBF0F00A490968B1FBF0F069
:1010200001F0DAFC48B9102C07D200222146501EEC
:1010300000F0BCF900206C6070BD012070BD0000A4
:1010400014000024000000242DE9F041044690F82B
:10105000A00015460F4601281DD0012684F8A06087
:10106000022084F8A10005EB850000EBC5003422C6
:1010700004EB80003830FFF7F4FA2A463946204660
:1010800004F0C6FF2068466284F8A160002084F85E
:10109000A000BDE8F0810220FBE7000070B504006D
:1010A00004D094F8A100002510B106E0012070BD25
:1010B000204684F8A05000F06BF8022084F8A100CC
:1010C0002068816921F070418161D4E901100143F8
:1010D000D4E903021043014320688269114381610E
:1010E0002068826829490A408260A08A0204206838
:1010F0008368A6693343134383602068C2680A404B
:10110000C260A08B02042068C368266A334313437D
:10111000C360206802690A400261A08C0204206852
:101120000369A66A334313430361206842690A4096
:101130004261A08D010420684269236B1A430A436F
:10114000426194F83500020294F8360001042068E8
:10115000C36A03F07F43C3622068C36A114394F8F3
:10116000346033430B43C3622068416B41F0060196
:1011700041632068816941F001018161C4F8A45094
:10118000012084F8A100002070BD000000F800F0EC
:101190002B4810B586B0016841F008010160006875
:1011A00000F00800059026481038016841F0100151
:1011B0000160006800F0100005902148001F0168E0
:1011C00041F480710160016801F48071059101684A
:1011D00041F400710160016801F40071059101683A
:1011E00041F48061016000680324694600F4806076
:1011F00005902020009001200190CDE902041148C3
:10120000FFF7E4FD4FF4E040009002200190002041
:101210006946CDE902040E2004900B48FFF7D6FD85
:1012200048F67C60009009486946FFF7CFFDFF2033
:10123000009007486946FFF7C9FD06B010BD0000E1
:10124000E4440258000402580020025800240258C6
:101250000028025870B5044690F8A0000E460128F8
:1012600020D0012584F8A050022084F8A10003EBCF
:10127000830000EBC30004EB80018E63086E3044F2
:10128000C1E90F02486E1044486438311A462046BE
:1012900004F0BEFE2068456284F8A150002084F866
:1012A000A00070BD022070BD70B5044690F8A0008B
:1012B0000E46012820D0012584F8A050022084F891
:1012C000A10003EB830000EBC30004EB8001886BFB
:1012D0003044C863086C10444864C1E9186238316E
:1012E0001A46204604F094FE2068456284F8A15016
:1012F000002084F8A00070BD022070BD134A417820
:101300001160111D03780A1DE3B143680B60017B76
:10131000C37A090741EA0361837A41EAC341437B07
:1013200041EA8341837B41EA4341C37B41EA034174
:10133000437A41EA0321037A007841EA43010143F9
:1013400011607047002008601060704798ED00E061
:10135000BFF35F8F0448016821F4803101600249C6
:10136000002070310860704724ED00E0074940F02C
:101370000100086005487038016841F4803101605F
:10138000BFF34F8FBFF36F8F7047000094ED00E005
:101390007047002809DB012100F01F02914040093D
:1013A000800000F1E020C0F8001170470E4BF0B44F
:1013B0001B68C3F30223C3F10704042C00D90424DF
:1013C0001D1D072D01D2002300E0DB1E012606FAB9
:1013D00004F56D1E0D409D409E40761E164045EA68
:1013E0000601F0BC06F067B90CED00E0064A00F01B
:1013F000070110684FF6FF03184040EA0120034937
:1014000008431060704700000CED00E00000FA0592
:1014100010B500F0B3FE084909684FF4807292FAE3
:10142000A2F201F47061B2FA82F2D140034A515C37
:10143000C8400349086010BD18440258DA7B000810
:101440000000002410B500F053FE0749096810227F
:1014500092FAA2F201F07001B2FA82F2D140034A8C
:10146000515CC84010BD000020440258DA7B0008DF
:10147000364930B50A68096812F00302344BC1F3EB
:1014800005311B68334C03F010032468DFED320A8A
:10149000B7EE001AC4F3CC0414FB03F300EE103AC9
:1014A0002E4BB8EE400A07D02D4C012A01D0022A5B
:1014B0004AD0B4FBF1F10BE0244C283C226895069D
:1014C000284A03D52468C4F3C104E240B2FBF1F119
:1014D00001EE901A1968B8EE612AC1F3080101EE15
:1014E000901A1968F8EE611A40EE201A31EE810A5E
:1014F00022EE000AC1F34621491C00EE901AF8EED4
:10150000600A80EE201AFCEEC10AC0ED000A1968DC
:10151000C1F30641491C00EE901AF8EE600A80EE15
:10152000201AFCEEC10AC0ED010A1968C1F3066178
:10153000491C00EE901AF8EE600A80EE201ABCEE0C
:10154000C10A80ED020A30BD074ABFE728440258AD
:101550002C4402583C4402580000003938440258D8
:1015600000093D000090D00340787D01364930B538
:101570000A68096812F00302344BC1F305511B6875
:10158000334C03F480732468DFED320AB7EE001A9F
:10159000C4F3CC0414FB03F300EE103A2E4BB8EE68
:1015A000400A07D02D4C012A01D0022A4AD0B4FBB0
:1015B000F1F10BE0244C283C22689506284A03D51B
:1015C0002468C4F3C104E240B2FBF1F101EE901AC9
:1015D0001968B8EE612AC1F3080101EE901A196882
:1015E000F8EE611A40EE201A31EE810A22EE000A6E
:1015F000C1F34621491C00EE901AF8EE600A80EE15
:10160000201AFCEEC10AC0ED000A1968C1F30641B8
:10161000491C00EE901AF8EE600A80EE201AFCEEEB
:10162000C10AC0ED010A1968C1F30661491C00EE48
:10163000901AF8EE600A80EE201ABCEEC10A80ED26
:10164000020A30BD074ABFE7284402582C4402581A
:1016500044440258000000394044025800093D004B
:101660000090D00340787D012DE9F84F04460068D2
:1016700000252E46010104F12400FE4FDFF8F88317
:1016800000901DD5606E50B1B0F5801F0CD0B0F544
:10169000001F0ED0B0F5401F1DD001250FE03868A7
:1016A00040F40030386016E00221201D04F020FED6
:1016B00003E00098022104F093FE05000BD02E46B3
:1016C0002088C00523D5606D05281ED2DFE800F014
:1016D0000C11161B1B00D8F80010626E21F440118B
:1016E0001143C8F80010EBE7386840F40030386068
:1016F00009E00021201D04F0FBFD03E0009800211B
:1017000004F06EFE05466DB100E001252E432088F1
:10171000800528D5A06D80281ED00CDC90B1402813
:101720000ED114E0D8F80010626D21F007011143CA
:10173000C8F80010EBE7C02813D0B0F5807F10D0B8
:1017400001250FE0386840F40030386009E00021DE
:10175000201D04F0CDFD03E00098002104F040FEC0
:10176000054685B12E432088DFF8109340052CD51F
:10177000D4F8A400B0F5800F20D00DDCA0B1B0F5F6
:10178000001F0FD115E0D8F80010A26D21F4E07110
:101790001143C8F80010E6E7B0F5C00F13D0B0F55C
:1017A000000F10D001250FE0386840F40030386099
:1017B00009E00021201D04F09BFD03E000980021BA
:1017C00004F00EFE054675B12E43208800052DD588
:1017D000D4F8A800B0F1007F21D00EDCA8B1B0F1A0
:1017E000807F10D116E0D9F80010D4F8A42021F49D
:1017F00060011143C9F80010E7E7B0F1407F13D052
:10180000B0F1806F10D001250FE0386840F400304F
:10181000386009E00021201D04F06AFD03E0009813
:10182000002104F0DDFD05466DB12E4320688001E6
:101830001FD5A06CD8B110280FD0202812D0302886
:1018400015D0012514E0D9F80010D4F8A82021F013
:10185000E0611143C9F80010E8E7386840F400304F
:10186000386004E00221201D04F042FD05466DB100
:101870002E432088C0042BD5E06DB0F5005F20D04A
:101880000DDCA0B1B0F5805F0FD115E07A48001FE4
:101890000168A26C21F0300111430160E9E7B0F565
:1018A000405F13D0B0F5804F10D001250FE03868AD
:1018B00040F40030386009E00021201D04F018FDDC
:1018C00003E00098002104F08BFD054685B12E430E
:1018D0002088800429D5206EB0F5403F23D010DC4D
:1018E00008B3B0F5803F14D0B0F5003F0FD115E03C
:1018F000D8F80010E26D21F4E0411143C8F800105F
:10190000E6E7B0F5802F0ED0B0F5A02F0BD0012563
:101910000AE00121201D04F0EBFC03E00098012106
:1019200004F05EFD05468DB12E43208840042AD583
:10193000D4F8AC00B0F1405F23D010DC08B3B0F1B4
:10194000805F14D0B0F1005F0FD115E0D8F800101F
:10195000226E21F4E0211143C8F80010E5E7B0F150
:10196000804F0ED0B0F1A04F0BD001250AE001212D
:10197000201D04F0BDFC03E00098012104F030FDBF
:1019800005466DB12E43208800041FD5E06ED8B106
:10199000B0F1805F0ED0B0F1005F10D0012514E0EF
:1019A000D9F80010D4F8AC2021F0E0411143C9F877
:1019B0000010E8E7386840F40030386004E00121A6
:1019C000201D04F095FC05466DB12E432068C00132
:1019D0001ED5606CD0B101280ED0022811D003288A
:1019E00014D0012513E0D8F80010E26E21F0405128
:1019F0001143C8F80010E9E7386840F40030386057
:101A000004E00221201D04F073FC054675B12E434D
:101A10002068DFF86CB040025AD51A48016841F4DA
:101A200080710160FFF7D4FA82460EE01248001F71
:101A30000168626C21F0030111430160E8E7FFF7E0
:101A4000C7FAA0EB0A0064283AD80E480068C0051F
:101A5000F5D5B5BB094818300068B4F8B01000F4EB
:101A6000407001F44071884219D004481830016870
:101A70000AE000002C4402585044025858440258CE
:101A80001044025800480258026821F4407142F4A0
:101A900080320260026822F4803202600160D4F871
:101AA000B000B0F5807F22D1FFF792FA824609E0BC
:101AB000FFF78EFAA0EB0A0141F28830814201D98A
:101AC000032504E0FE4800688007F1D57DB12E4370
:101AD0002078DFF8F0A3C0073CD0A06F182837D0DB
:101AE00025DC78B3082828D0102824D12BE0D4F89E
:101AF000B000C0F3012103290ED0DBF8001021F45F
:101B00007C51CBF80010EE480168B4F8B020C2F365
:101B10000B0211430160DBE7DBF80020EA4B22F403
:101B20007C5203EA10100243CBF80020EBE7202898
:101B30000ED028280CD001250BE00121201D04F037
:101B4000D7FB04E004E00098012104F049FC0546BD
:101B50005DB12E43207880071ED5606F062819D20C
:101B6000DFE800F0160C11161616DAF80010A26F56
:101B700021F038011143CAF80010EBE70121201DC4
:101B800004F0B6FB03E00098012104F029FC0546AF
:101B900075B100E001252E43207840071FD5D4F809
:101BA0009000062819D2DFE800F0160C1116161660
:101BB000DAF80010626F21F007011143CAF8001033
:101BC000EAE70121201D04F093FB03E000980121C6
:101BD00004F006FC05469DB100E001252E43207867
:101BE00080062BD5D4F88C00B0F1405F24D011DCF6
:101BF00010B3B0F1805F15D0B0F1005F10D116E0E6
:101C0000D9F80010D4F8902021F007011143C9F849
:101C10000010E4E7B0F1804F0ED0B0F1A04F0BD030
:101C200001250AE00021201D04F062FB03E000987A
:101C3000022104F0D5FB05468DB12E4320784006E5
:101C40002BD5D4F89800B0F5406F24D011DC10B338
:101C5000B0F5806F15D0B0F5006F10D116E0DAF84E
:101C60000010D4F88C2021F0E0411143CAF8001094
:101C7000E4E7B0F5805F0ED0B0F5A05F0BD0012592
:101C80000AE00021201D04F033FB03E0009802214C
:101C900004F0A6FB05468DB12E43207800062BD517
:101CA000D4F89C00B0F5C04F24D011DC10B3B0F5CF
:101CB000005F15D0B0F5804F10D116E0D9F80010B4
:101CC000D4F8982021F4E0511143C9F80010E4E75A
:101CD000B0F5004F0ED0B0F5204F0BD001250AE033
:101CE0000021201D04F004FB03E00098022104F011
:101CF00077FB054665B32E43207800070BD5D4F853
:101D00008000B0F5805F2DD0DAF8002022F4405238
:101D10000243CAF800202078C0060BD5D4F89400FE
:101D2000B0F5807F24D0D9F8002022F4407202431D
:101D3000C9F80020206800032CD5D4F8A000E8B131
:101D4000B0F5803F1FD0B0F5003F21D0012520E045
:101D5000D9F80010D4F89C2021F460411143C9F84F
:101D60000010C9E70098022104F03AFB0643D2E7CD
:101D70000098022104F034FB0643DBE70021201D1C
:101D800004F0B6FA03E00098022104F029FB0546AE
:101D900085B12E432068400322D5D4F88400B0F5E5
:101DA000801F11D0B0F5001F13D0B0F5401F15D023
:101DB000012514E0D9F80010D4F8A02021F4403116
:101DC0001143C9F80010E5E7386840F40030386086
:101DD00004E00098012104F003FB054655B12E43B1
:101DE0002068C0031CD5E06C70B1B0F5803F10D006
:101DF000012514E0DAF80010D4F8842021F4401111
:101E00001143CAF80010EBE7386840F4003038603E
:101E100004E00221201D04F06BFA0546C5B12E43F3
:101E20002068800004D50098022104F0D9FA064306
:101E3000206880031BD5E06FB8B1B0F5807F10D06B
:101E4000B0F5007F11D0B0F5407F0ED001250DE038
:101E50001C4808380168E26C21F4803111430160AC
:101E6000DEE7386840F40030386045B32E43206820
:101E7000C00207D5D8F80000226F20F000401043C0
:101E8000C8F800002068C00008D5DBF80010D4F8BE
:101E9000B42021F480411143CBF800102068800267
:101EA00007D5D8F80010A26E21F080711143C8F850
:101EB00000102068400014D5DBF8001006E01EE09A
:101EC0007044025854440258CFFFFF0021F40041EF
:101ED000CBF80010DBF80010D4F8B8201143CBF891
:101EE00000102068002806DA0A480168226D21F0F7
:101EF0004051114301605EB10120BDE8F88FDAF86E
:101F00000010E26F21F440711143CAF80010AEE7EF
:101F10000020F2E74C4402582DE9F047DFF8BC916D
:101F200004460E46D9F8000000F00700B0420CD27B
:101F3000D9F8001021F007013143C9F80010D9F891
:101F4000000000F00700B0427ED12078DFF89081D9
:101F5000800707D5D8F80010E26821F00F0111437F
:101F6000C8F800102078C00762D0D8F80010A26826
:101F700021F470611143C8F800105949606818399C
:101F800002281CD003281DD0096801281DD049074C
:101F9000002960DA524F083F396821F007010143F8
:101FA0003960FFF715F80546606841F2883102286C
:101FB00013D003281ED001288A4627D034E00968B0
:101FC0008903E5E709688901E2E7C905E0E7FEF76B
:101FD000FFFF411B514501D923E08A463868C0F311
:101FE000C2000228F3D123E0FEF7F2FF411B514566
:101FF00001D916E08A463868C0F3C2000328F3D13D
:1020000016E0FEF7E5FF411B51450AD83868C0F3DA
:10201000C2000128F5D10BE0FEF7DAFF411B514564
:1020200002D90320BDE8F087386810F0380FF3D1EB
:10203000D9F80010484601F00701B1420DD90168F6
:1020400021F00701314300E005E00160006800F085
:102050000700B04201D00120E4E72078400707D50F
:10206000D8F80010226921F070011143C8F800105F
:10207000207801071B4805D50168626921F07001CD
:10208000114301602178C90605D50168A26921F4D0
:10209000E061114301602078800607D51149091DD0
:1020A0000868E26920F070001043086000F066F8EC
:1020B000D8F800104FF4807292FAA2F201F4706125
:1020C000B2FA82F2D140084A515CC8400749086020
:1020D0000F20FEF799FF0020A4E700000020005227
:1020E000184402581C440258DA7B000800000024FF
:1020F00010B5FFF78DF908490968012292FAA2F29A
:1021000001F00F01B2FA82F2D140044A515CC8409A
:102110000349086010BD000018440258DA7B00082B
:102120000400002410B5FFF7E3FF074909681022F7
:1021300092FAA2F201F07001B2FA82F2D140034A9F
:10214000515CC84010BD00001C440258DA7B0008F6
:1021500010B5FFF7CDFF074909684FF4807292FA76
:10216000A2F201F4E061B2FA82F2D140024A515C7B
:10217000C84010BD1C440258DA7B00083548F0B551
:102180000068364D10F03801334809D00411082991
:1021900004D0334E10290BD018290BD02046F0BDA7
:1021A00029688906FBD52968C1F3C101C840F0BD83
:1021B0003046F0BD274918310A68096812F0030259
:1021C000284BC1F305111B68274F03F001033F683B
:1021D000DFED260AB7EE001AC7F3CC0717FB03F3AF
:1021E00000EE103A224BB8EE400A06D0012A01D088
:1021F000022A2BD0B4FBF1F008E02A68920603D53E
:102200002A68C2F3C102D040B0FBF1F001EE900A9F
:102210001868B8EE612AC0F3080001EE900A186849
:10222000F8EE611A40EE201A31EE810A22EE000A21
:10223000C0F34620401C00EE900AF8EE600A80EEE3
:10224000201ABCEEC10A10EE100AF0BDB6FBF1F088
:10225000DCE70000104402580090D003004402580C
:1022600040787D012C440258344402580000003963
:10227000304402582DE9F05F04460078DFF8FC8313
:1022800041F28839DFF8F8A3FE4DC0074ED0D8F8E8
:1022900000104046C1F3C20102291AD00068C0F301
:1022A000C200032805D1DAF8000000F0030002287C
:1022B0000FD06068B0F5803F12D010B1B0F5A02FFC
:1022C00019D0286820F480302860286820F4802005
:1022D00009E02868800329D56068002874D025E0CB
:1022E000286840F480302860606890B1FEF770FE86
:1022F00006464F4609E0286840F480202860EFE752
:10230000FEF766FE801BB8427DD828688003F7D5AB
:102310000CE0FEF75DFE06464F4604E0FEF758FE71
:10232000801BB842F0D828688003F7D42078D64FB5
:1023300080075AD5D8F8001040464FF47C3B11F086
:10234000380F13D00068C0F3C200032803D1DAF8B5
:10235000000080070AD0E068A8B3296821F01901BD
:1023600001432960FEF734FE06461DE02868400759
:1023700002D5E0680028B1D02868E16820F0190093
:1023800008432860FEF724FE064604E0FEF720FE20
:10239000801B0228B8D828684007F7D507E0FEF769
:1023A00017FE801B0228AFD828684007F7D5386889
:1023B0009BFAABF220F47C312069B2FA82F29040B1
:1023C0000143396011E000E0AEE0286820F0010030
:1023D0002860FEF7FDFD064604E0FEF7F9FD801BD0
:1023E000022891D828684007F7D42078C00655D530
:1023F000D8F8001040464FF0F84BC1F3C201012954
:1024000017D0006800E0EDE0C0F3C200032805D15A
:10241000DAF8000000F0030001280AD0E069002883
:1024200028682CD040F080002860FEF7D1FD0646D9
:1024300016E02868C00502D5E069802874D13868A4
:102440009BFAABF220F0F841206AB2FA82F2904097
:102450000143396022E0FEF7BBFD801B022899D8BA
:102460002868C005F7D538689BFAABF2216AB2FA42
:1024700082F220F0F8409140084338600EE020F0EE
:1024800080002860FEF7A4FD064604E0FEF7A0FDEC
:10249000801B022887D82868C005F7D42078000759
:1024A00024D5774F60694C37002838680FD040F04A
:1024B00001003860FEF78CFD064604E0FEF788FD5B
:1024C000801B02288DD838688007F7D50EE020F0F1
:1024D00001003860FEF77CFD064604E0FEF778FD5B
:1024E000801B02287ED838688007F7D420788006C1
:1024F00023D5A069002828680FD040F480502860B8
:10250000FEF766FD064604E0FEF762FD801B02282A
:1025100068D828688004F7D50FE020F48050286040
:10252000FEF756FD064605E0D6E0FEF751FD801B9E
:10253000022857D828688004F7D42078400744D56B
:10254000524F386840F480703860FEF741FD06460F
:1025500004E0FEF73DFD801B642843D83868C005C1
:10256000F7D5474FA068483701280AD008B1052899
:1025700011D0386820F001003860386820F004007D
:1025800002E0386840F001003860A06888B1FEF7CA
:102590001FFD064609E0386840F004003860F0E7A7
:1025A000FEF716FD811B49451CD838688007F7D512
:1025B0000BE0FEF70DFD064604E0FEF709FD811B6A
:1025C00049450FD838688007F7D4606AF0B3D8F867
:1025D0000010C1F3C20103297ED00228286820F030
:1025E000807000E079E0286003D0FEF7F1FC04463B
:1025F00087E0FEF7EDFC064604E0FEF7E9FC801BF1
:1026000002287BD828688001F7D4DAF8001040F25D
:10261000F3329143E26A41EA0211A26A1143CAF815
:10262000001094F834004FF4FE02218E4002491E3F
:10263000A0F5007080B2C1F308010843218F491E44
:1026400002EA0141084394F83C1000E05CE0491EB6
:10265000120202EA016108430949083108600B1DB2
:1026600019684FF6F872A06C914392FAA2F2B2FA8E
:1026700082F2904001431960014809E01044025879
:1026800028440258004402580444025800480258A2
:10269000001D0168226C21F00C01114301600168EA
:1026A000626C21F0020111430160016841F4803144
:1026B0000160016841F400310160016841F480214A
:1026C0000160016841F001010160286840F08070FC
:1026D0002860FEF77DFC01E018E00FE0044604E00E
:1026E000FEF776FC001B022808D828688001F7D581
:1026F0000AE0FEF76DFC001B022802D90320BDE8AA
:10270000F09F28688001F4D40020F8E70120F6E764
:1027100070B504000D4603D094F82C0010B107E00A
:10272000012070BD002084F82D00204600F018F82C
:10273000022084F82C002068211DFEF719FAD4E944
:1027400000022946FEF754FA0448016841F00041AE
:102750000160012084F82C00002070BD0040005270
:10276000444800B587B0016841F00201016000688B
:1027700000F0020005903F482038016841F4805184
:102780000160006800F4805005903A4814380168F0
:1027900041F004010160016801F004010591016844
:1027A00041F008010160016801F00801059101682C
:1027B00041F010010160016801F01001059101680C
:1027C00041F020010160016801F0200105910168DC
:1027D00041F040010160016801F04001059101688C
:1027E00041F080010160016801F0800105910168FC
:1027F00041F4807101600068694600F480700590C2
:102800000D200090022001900120029003200390EF
:102810000C2004901848FEF7D9FA4CF2037000908F
:1028200016486946FEF7D2FA4FF6837000901448B6
:102830006946FEF7CBFA4FF63F0000901148694613
:10284000FEF7C4FA48F2371000900F486946FEF7C9
:10285000BDFA4FF47F4000900C486946FEF7B6FA87
:1028600040F2FF6000900A486946FEF7AFFA07B0F1
:1028700000BD0000F444025800080258000C025841
:10288000001002580014025800180258001C025888
:102890000020025810B5044690F82C00022809D0F8
:1028A000022084F82C002068FEF78AF9012084F8C1
:1028B0002C00002010BD70B5044690F82C000D4689
:1028C00002280CD0022084F82C002068FEF77EF944
:1028D0002868022804D0012084F82C00002070BD54
:1028E0000520F9E770B5040015460E4603D094F8AC
:1028F000450010B107E0012070BD002084F84400BD
:10290000204600F021F8206804F10801FEF7C6F81F
:10291000A26831462068FEF7FDF8E36A2946D4E94B
:102920000102FEF79BF8A168206850F8212042F0D0
:10293000010240F821200348016841F00041016094
:10294000002070BD004000521A4800B587B00168F1
:1029500041F480510160006800F4805005901548F2
:102960000C30016841F008010160016801F00801C4
:102970000591016841F0100101600068694600F0AE
:10298000100005904EF2B3700090022001900120DB
:102990000290032003900C2004900748FEF716FADB
:1029A0004FF68070009005486946FEF70FFA07B0B1
:1029B00000BD0000D4440258000C02580010025818
:1029C0004FF0E0210428086903D020F004000861DA
:1029D000704740F00400FAE7401EB0F1807F10B568
:1029E00001D3012010BD4FF0E02460610F2160177A
:1029F00004F061FE0020A06107202061002010BDCE
:102A00007047704790F8791090F87A000843704743
:102A100070B502680446D0691368916810F00F0F12
:102A200064D0594D03F490760D40354376D0C507F8
:102A300007D0DD0505D501251562E26F42F00102E0
:102A4000E267820708D5CA0706D0256802222A62F3
:102A5000E26F42F00402E267420708D5CA0706D0D7
:102A6000256804222A62E26F42F00202E26702074E
:102A70000ED503F0200201F080552A4352EAC172BC
:102A800006D0256808222A62E26F42F00802E26757
:102A9000E26F002A3AD0800608D503F0200001F04A
:102AA0008051084302D0204604F0E6FAE06F0007A8
:102AB00003D42068806840062AD5204604F0CEFA68
:102AC0002068816849061ED5816821F04001816037
:102AD000606FC0B12D490165606FFEF725F90028D0
:102AE00014D0606F016DBDE870400847850615D5AC
:102AF00003F0200501F0805635430FD02046BDE895
:102B0000704004F0B9BA2046FFF77BFF70BD05E0C6
:102B10002046FFF776FF0020E067F7E7C6024FF098
:102B200020050CD54E020AD5E803106284F87950CE
:102B300084F87A502046BDE87040FFF761BF060672
:102B40000AD503F0800601F400010E4304D02046AC
:102B5000BDE8704004F020BD41060BD5590609D5EB
:102B60001168204621F04001116084F8795000F08E
:102B700005F9CBE70002C9D55800C7D5106820F089
:102B800080401060C2E7000001000010497000089A
:102B900010B5040003D094F8790010B107E00120CB
:102BA00010BD002084F87800204600F027F824208B
:102BB00084F879002068016821F001010160204655
:102BC00004F096FA0128EBD0606B10B1204604F0B7
:102BD000A9F92068416821F490414160206881682A
:102BE00021F02A0181602068016841F00101016043
:102BF0002046BDE8104004F0F9B9000010B50068A7
:102C000086B01B49884230D11A48016841F0010161
:102C10000160006800F0010005901648103001685E
:102C200041F01001016000680121134C00F0100018
:102C300005904FF4007000900220CDE9010103904F
:102C40000720694604902046FEF7C0F84FF48061E3
:102C5000204600916946FEF7B9F82520FEF799FB5A
:102C6000032225201146FEF7A1FB06B010BD00008F
:102C700000100140E04402580000025890F87A30F9
:102C8000202B4CD1B9B1B2B190F87830012B46D09D
:102C9000012380F878304166A0F86820A0F86A2007
:102CA000FF228168B1F5805F07D07F2351B1B1F178
:102CB000805F0CD010E001207047016921B940F21B
:102CC000FF1107E0016909BBA0F86C2004E001696D
:102CD000E1B13F21A0F86C100021C167222280F8E9
:102CE0007A2080F8781001688A6842F001028A60D0
:102CF00001680A6892000CD50A6842F480720A6082
:102D00000068816841F08051816006E0A0F86C3075
:102D1000E2E7086840F490700860002070470220E5
:102D20007047000030B50068114988420CD1114A43
:102D30005088010408D411464FF000034404097878
:102D400006D50A2901D0538030BD40F400400DE083
:102D50000D2909D0084DC0F30D04401C80B2C728CE
:102D600029555080EFD830BD40F48040508030BDB0
:102D7000001001400C0000247C0000247047FEE796
:102D80001B4870B586B0016841F00101016001681F
:102D900001F001010591016841F004010160016841
:102DA00001F004010591016841F0800101600068B3
:102DB00003240025694600F08000059002200126CA
:102DC000CDE902040B48CDE90065FDF7FFFF700374
:102DD00003948DE8610008486946FDF7F7FF0C2071
:102DE000009006486946FDF7F1FF06B070BD00008F
:102DF000E04402580000025800080258001C025823
:102E00002DE9F0470126304CDFF8C080DFF8C09094
:102E10007703304D01281DD02078A0B10821284625
:102E2000FEF7C8F8C0B104212846FEF7C3F898B1F0
:102E300039464046FEF7BEF870B101214846FEF71C
:102E4000B9F8012808D008212846FEF7B3F8012870
:102E500026D037E02670E1E70A2004F047FC002086
:102E6000207008212846FEF7A5F880B104212846E5
:102E7000FEF7A0F870B139464046FEF79BF858B10E
:102E800001214846FEF796F8012807D01AE00120F4
:102E9000BDE8F0870220FBE70320F9E70420F7E70D
:102EA00004212846FEF786F801280BD13946404612
:102EB000FEF780F8012805D101214846FEF77AF88F
:102EC00000B926700020E3E7200000240008025823
:102ED00000000258001C02580E490F4A70B5064601
:102EE00008881268002422B13046BDE8704002F024
:102EF000C3BD4D8800214543084602F017FC02F08F
:102F000083FDB1B2054801E00180641CAC42FBD3F3
:102F100070BD000010020024FC02002400000860C4
:102F20002DE9F05F394C3A4DA071296839B102F0B2
:102F3000C7FDE88A2080288B6080BDE8F09F334978
:102F40002C232A254FF0F0092B2649F2413A4FF461
:102F5000305E45F2105B89884FF448774FF4A078D3
:102F600045F2103C4FF4F07258B1A4F8008051457E
:102F7000A4F8029001D0614529D123816581A68101
:102F800039E0A4F800905145A4F8028001D06145D1
:102F900008D1238161456581A68131D1A4F80080E3
:102FA00062802DE0594508D1A4F808E04FF428507C
:102FB00060814FF42C50A08106E0A1F5C850633821
:102FC0001ED123816681A5812280678018E0594542
:102FD00008D1A4F808E04FF4285060814FF42C5039
:102FE000A08106E0A1F5C850633804D12381658132
:102FF000A68127806280614502D12280A4F80280E8
:103000000020BDE8F05F02F0B5BA00001002002415
:10301000FC0200242DE9F04104463A480D460068C0
:1030200020B12046BDE8F04102F05EBD364E270AD1
:103030004FEA15283146B0884989A0F51343413B32
:103040000CD0A0F5A643103B08D0A0F5AA43103B36
:1030500011D0A0F5C853633B27D04BE0084602F0DF
:10306000C7FC384602F0B8FCE0B202F0B5FCB0890B
:1030700002F0BEFC38E0084602F0BAFC384602F026
:10308000ABFC7089401C80B202F0B2FCE0B202F0EE
:10309000A3FCB08902F0ACFC404602F09DFCB08974
:1030A000401C80B202F0A4FC21E0B07918B930884D
:1030B000001B401E84B2084602F09AFC270A3846DC
:1030C00002F08AFCE0B202F087FC384602F084FC91
:1030D000E0B202F081FCB08902F08AFC404602F0C6
:1030E0007BFCE8B202F078FC404602F075FCE8B2E6
:1030F00002F072FC054930890880881C0280BDE816
:10310000F0810000FC02002410020024FEFF076092
:103110002DE9F04F95B002F01DFFFE4D4FF6FF7AFE
:1031200049F2413945F21036A5F14C0845F21054E8
:1031300041F66317A88018B102F04AFD02F08DB97C
:10314000F548016841F00201016000680EA900F035
:103150000200139020200E9001200F901090032069
:103160001190EE48FDF732FE02F0A4F9EC4910226E
:10317000C8F800104046EB49C8F804100021C8F810
:103180000810C8F80C10C0E904121202C8F8181090
:10319000C8F81C10C0E908129200C0E90A12920196
:1031A000C8F830101120C8E90D12CDE907015520EB
:1031B000099015200290CDE90001D6486A460D918C
:1031C0004C38069107A9FFF78DFB322004F08EFAE8
:1031D000D32002F00DFC02F099F9A88002F096F9D4
:1031E000A88002F093F90AEA00205246A88002F073
:1031F0008DF9A9880843A880484546D0D42002F01C
:10320000F7FB02F083F9A88002F080F9A88002F0B1
:103210007DF902EA0020A88002F078F9A988084325
:10322000A880B04231D04FF45A4002F0E1FB02F0E6
:103230006DF9A8804FF45B4002F0DAFB02F066F90A
:1032400002EA0020A8804FF45C4002F0D1FB02F0BB
:103250005DF9A9880843A880B0F5004F7DD0A04251
:1032600013D0A12002F0C4FB02F050F9A88002F0B4
:103270004DF902EA0020A88002F048F9A988084325
:10328000A880A0F5AE41613968D080B2484566D1CA
:10329000CF2002F0ADFB002002F09EFBC12002F027
:1032A0009BFB302002F098FBED2002F0A1FB642094
:1032B00002F092FB032002F08FFB122002F08CFB45
:1032C000812002F089FBE82002F092FB852002F0C9
:1032D00083FB102002F080FB7A2002F07DFBCB20E4
:1032E00002F086FB392002F077FB2C2002F074FB01
:1032F000002002F071FB342002F06EFB022002F08D
:103300006BFBF72002F074FB202002F065FBEA2043
:1033100002F06EFB002002F05FFB002002F05CFB7D
:10332000C02002F065FB1B2002F056FBC12002F01A
:103330005FFB012002F050FBC52002F059FB30205A
:1033400002F04AFB302002F047FBC72002F050FB9E
:10335000B72002F041FB362002E0B4E0B0E0B4E078
:1033600002F046FB482002F037FB3A2002F040FB17
:10337000552002F031FBB12002F03AFB002002F0B0
:103380002BFB1A2002F028FBB62002F031FB0A20AA
:1033900002F022FBA22002F01FFBF22002F028FB29
:1033A000002002F019FB262002F022FB012002F08F
:1033B00013FBE02002F01CFB0F2002F00DFB2A2083
:1033C00002F00AFB282002F007FB082002F004FBB1
:1033D0000E2002F001FB082002F0FEFA542002F059
:1033E000FBFAA92002F0F8FA432002F0F5FA0A20CD
:1033F00002F0F2FA0F2002F0EFFA002002F0ECFAED
:10340000002002F0E9FA002002F0E6FA002002F0C3
:10341000E3FAE12002F0ECFA002002F0DDFA1520D8
:1034200002F0DAFA172002F0D7FA072002F0D4FAF5
:10343000112002F0D1FA062002F0CEFA2B2002F081
:10344000CBFA562002F0C8FA3C2002F0C5FA05205B
:1034500002F0C2FA102002F0BFFA0F2002F0BCFA0C
:103460003F2002F0B9FA3F2002F0B6FA0F2002F036
:10347000B3FA2B2002F0BCFA002002F0ADFA0020D3
:1034800002F0AAFA012002F0A7FA3F2002F0A4FA03
:103490002A2002F0ADFA002002F09EFA002002F08D
:1034A0009BFA002002F098FAEF2002F095FA112022
:1034B00002F09EFA782004F019F9292001F010BFDB
:1034C000AF8001F012BFAC80FDE3B0427ED1ED20B1
:1034D00002F08EFA012002F07FFAFE2002F07CFA60
:1034E000EE2002F085FADE2002F076FA212002F0CA
:1034F00073FAF12002F07CFA012002F06DFADF206D
:1035000002F076FA102002F067FAC42002F070FA96
:103510008F2009E010020024E04402580004025801
:10352000004000520441005202F056FAC62002F058
:103530005FFA002002F050FAE22002F04DFAE22099
:1035400002F04AFAE22002F047FABF2002F050FAF5
:10355000AA2002F041FAB02002F04AFA0D2002F04F
:103560003BFA002002F038FA0D2002F035FA002074
:1035700002F032FA112002F02FFA002002F02CFAA9
:10358000192002F029FA002002F026FA212002F088
:1035900023FA002002F020FA2D2002F01DFA00206C
:1035A00002F01AFA3D2002F017FA002002F014FA95
:1035B0005D2002F011FA002002F00EFA5D2002F008
:1035C0000BFA002002F008FAB12000E0FEE302F05E
:1035D0000FFA802002F000FA002002F0FDF98B20A3
:1035E00002F0FAF9002002F0F7F9962002F0F4F95F
:1035F000002002F0F1F9B22002F0FAF9002002F006
:10360000EBF9002002F0E8F9022002F0E5F90020D1
:1036100002F0E2F9032002F0DFF9002002F0DCF909
:10362000B32002F0E5F9002002F0D6F9002002F004
:10363000D3F9002002F0D0F9002002F0CDF90020EB
:1036400002F0CAF9002002F0C7F9002002F0C4F924
:10365000002002F0C1F9002002F0BEF9002002F0C3
:10366000BBF9002002F0B8F9002002F0B5F9002003
:1036700002F0B2F9002002F0AFF9002002F0ACF93C
:10368000002002F0A9F9002002F0A6F9002002F0C3
:10369000A3F9002002F0A0F9002002F09DF900201B
:1036A00002F09AF9002002F097F9002002F094F954
:1036B000002002F091F9B42002F09AF98B2002F078
:1036C0008BF9002002F088F9962002F085F900209D
:1036D00002F082F9A12002F07FF9002002F07CF9CB
:1036E000B52002F085F9022002F076F9002002F000
:1036F00073F9032002F070F9002002F06DF9042044
:1037000002F06AF9002002F067F9B62002F070F9C1
:10371000002002F061F9002002F05EF9B72002F00B
:1037200067F9002002F058F9002002F055F93F2017
:1037300002F052F9002002F04FF95E2002F04CF93D
:10374000002002F049F9642002F046F9002002F05E
:1037500043F98C2002F040F9002002F03DF9AC2042
:1037600002F03AF9002002F037F9DC2002F034F9D7
:10377000002002F031F9702002F02EF9002002F052
:103780002BF9902002F028F9002002F025F9EB2017
:1037900002F022F9002002F01FF9DC2002F01CF9EF
:1037A000002002F019F9B82002F022F9002002F0FE
:1037B00013F9002002F010F9002002F00DF90020AA
:1037C00002F00AF9002002F007F9002002F004F9E3
:1037D000002002F001F9002002F0FEF8BA2002F009
:1037E00007F9242002F0F8F8002002F0F5F8002094
:1037F00002F0F2F8002002F0EFF8C12002F0F8F831
:10380000202002F0E9F8002002F0E6F8542002F04F
:10381000E3F8002002F0E0F8FF2002F0DDF80020DD
:1038200002F0DAF8C22002F0E3F80A2002F0D4F83D
:10383000002002F0D1F8042002F0CEF8002002F0BF
:10384000CBF8C32002F0D4F83C2002F0C5F80020E9
:1038500002F0C2F83A2002F0BFF8002002F0BCF8F3
:10386000392002F0B9F8002002F0B6F8372002F053
:10387000B3F8002002F0B0F83C2002F0ADF80020D0
:1038800002F0AAF8362002F0A7F8002002F0A4F80F
:10389000322002F0A1F8002002F09EF82F2002F062
:1038A0009BF8002002F098F82C2002F095F80020F8
:1038B00002F092F8292002F08FF8002002F08CF834
:1038C000262002F089F8002002F086F8242002F079
:1038D00083F8002002F080F8242002F07DF8002018
:1038E00002F07AF8232002F077F8002002F074F852
:1038F0003C2002F071F8002002F06EF8362002F051
:103900006BF8002002F068F8322002F065F8002021
:1039100002F062F82F2002F05FF8002002F05CF85D
:103920002C2002F059F8002002F056F8292002F06D
:1039300053F8002002F050F8262002F04DF8002045
:1039400002F04AF8242002F047F8002002F044F880
:10395000242002F041F8002002F03EF8232002F07B
:103960003BF8002002F038F8C42002F041F8622051
:1039700002F032F8002002F02FF8052002F02CF8B7
:10398000002002F029F8842002F026F8002002F03E
:1039900023F8F02002F020F8002002F01DF8182093
:1039A00002F01AF8002002F017F8A42002F014F830
:1039B000002002F011F8182002F00EF8002002F0AA
:1039C0000BF8502002F008F8002002F005F80C2057
:1039D00002F002F8002001F0FFFF172001F0FCFFC9
:1039E000002001F0F9FF952001F0F6FF002001F022
:1039F000F3FFF32001F0F0FF002001F0EDFFE620DF
:103A000001F0EAFF002001F0E7FFC52001F0F0FF20
:103A1000322001F0E1FF002001F0DEFF442001F040
:103A2000DBFF002001F0D8FF652001F0D5FF00206A
:103A300001F0D2FF762001F0CFFF002001F0CCFF93
:103A4000882001F0C9FF002001F0C6FFC62001F068
:103A5000CFFF202001F0C0FF002001F0BDFF1720A4
:103A600001F0BAFF002001F0B7FF012001F0B4FF20
:103A7000002001F0B1FFC72001F0BAFF002001F0E3
:103A8000ABFF002001F0A8FF002001F0A5FF0020FF
:103A900001F0A2FFC82001F0ABFF002001F09CFF65
:103AA000002001F099FF002001F096FF002001F0B6
:103AB00093FFC92001F09CFF002001F08DFF002042
:103AC00001F08AFF002001F087FF002001F084FF51
:103AD000002001F081FF002001F07EFF002001F0B6
:103AE0007BFF002001F078FF002001F075FF00202F
:103AF00001F072FF002001F06FFF002001F06CFF69
:103B0000002001F069FF002001F066FF002001F0B5
:103B100063FF002001F060FFE02001F069FF162044
:103B200001F05AFF002001F057FF1C2001F054FF64
:103B3000002001F051FF212001F04EFF002001F094
:103B40004BFF362001F048FF002001F045FF4620E2
:103B500001F042FF002001F03FFF522001F03CFF46
:103B6000002001F039FF642001F036FF002001F051
:103B700033FF7A2001F030FF002001F02DFF8B2071
:103B800001F02AFF002001F027FF992001F024FF17
:103B9000002001F021FFA82001F01EFF002001F00D
:103BA0001BFFB92001F018FF002001F015FFC42011
:103BB00001F012FF002001F00FFFCA2001F00CFFFE
:103BC000002001F009FFD22001F006FF002001F0E3
:103BD00003FFD92001F000FF002001F0FDFEE020EE
:103BE00001F0FAFE002001F0F7FEF32001F0F4FEF0
:103BF000002001F0F1FEE12001F0FAFE162001F0B4
:103C0000EBFE002001F0E8FE1C2001F0E5FE0020A4
:103C100001F0E2FE222001F0DFFE002001F0DCFED8
:103C2000362001F0D9FE002001F0D6FE452001F03B
:103C3000D3FE002001F0D0FE522001F0CDFE002086
:103C400001F0CAFE642001F0C7FE002001F0C4FEAE
:103C50007A2001F0C1FE002001F0BEFE8B2001F0B1
:103C6000BBFE002001F0B8FE992001F0B5FE002057
:103C700001F0B2FEA82001F0AFFE002001F0ACFE82
:103C8000B92001F0A9FE002001F0A6FEC42001F039
:103C9000A3FE002001F0A0FECA2001F09DFE00203E
:103CA00001F09AFED22001F097FE002001F094FE70
:103CB000D82001F091FE002001F08EFEE02001F0FE
:103CC0008BFE002000E08BE301F086FEF32001F084
:103CD00083FE002001F080FEE22001F089FE052035
:103CE00001F07AFE002001F077FE0B2001F074FE57
:103CF000002001F071FE1B2001F06EFE002001F09B
:103D00006BFE342001F068FE002001F065FE4420C7
:103D100001F062FE002001F05FFE4F2001F05CFE2A
:103D2000002001F059FE612001F056FE002001F054
:103D300053FE792001F050FE002001F04DFE882056
:103D400001F04AFE002001F047FE972001F044FEFA
:103D5000002001F041FEA62001F03EFE002001F00F
:103D60003BFEB72001F038FE002001F035FEC220F6
:103D700001F032FE002001F02FFEC72001F02CFEE2
:103D8000002001F029FED12001F026FE002001F0E4
:103D900023FED62001F020FE002001F01DFEDD20D4
:103DA00001F01AFE002001F017FEF32001F014FECE
:103DB000002001F011FEE32001F01AFE052001F0C1
:103DC0000BFE002001F008FE0A2000E006E301F0EF
:103DD00003FE002001F000FE1C2001F0FDFD00208C
:103DE00001F0FAFD332001F0F7FD002001F0F4FDB1
:103DF000442001F0F1FD002001F0EEFD502001F023
:103E0000EBFD002001F0E8FD622001F0E5FD00205F
:103E100001F0E2FD782001F0DFFD002001F0DCFD83
:103E2000882001F0D9FD002001F0D6FD972001F097
:103E3000D3FD002001F0D0FDA62001F0CDFD002033
:103E400001F0CAFDB72001F0C7FD002001F0C4FD5C
:103E5000C22001F0C1FD002001F0BEFDC72001F02D
:103E6000BBFD002001F0B8FDD12001F0B5FD002020
:103E700001F0B2FDD52001F0AFFD002001F0ACFD56
:103E8000DD2001F0A9FD002001F0A6FDF32001F0E6
:103E9000A3FD002001F0A0FDE42001F0A9FD012018
:103EA00001F09AFD002001F097FD012001F094FD42
:103EB000002001F091FD022001F08EFD002001F0B4
:103EC0008BFD2A2001F088FD002001F085FD3C20BB
:103ED00001F082FD002001F07FFD4B2001F07CFD10
:103EE000002001F079FD5D2001F076FD002001F059
:103EF00073FD742001F070FD002001F06DFD842041
:103F000001F06AFD002001F067FD932001F064FDDF
:103F1000002001F061FDA22001F05EFD002001F013
:103F20005BFDB32001F058FD002001F055FDBE20DF
:103F300001F052FD002001F04FFDC42001F04CFDC6
:103F4000002001F049FDCD2001F046FD002001F0E8
:103F500043FDD32001F040FD002001F03DFDDD20B8
:103F600001F03AFD002001F037FDF32001F034FDAF
:103F7000002001F031FDE52001F03AFD002001F0C4
:103F80002BFD002001F028FD002001F025FD002080
:103F900001F022FD022001F01FFD002001F01CFDB8
:103FA000292001F019FD002001F016FD3C2001F050
:103FB00013FD002001F010FD4B2001F00DFD00204D
:103FC00001F00AFD5D2001F007FD002001F004FD75
:103FD000742001F001FD002001F0FEFC842001F0BE
:103FE000FBFC002001F0F8FC932001F0F5FC002020
:103FF00001F0F2FCA22001F0EFFC002001F0ECFC4B
:10400000B32001F0E9FC002001F0E6FCBE2001F045
:10401000E3FC002001F0E0FCC42001F0DDFC002006
:1040200001F0DAFCCD2001F0D7FC002001F0D4FC37
:10403000D32001F0D1FC002001F0CEFCDC2001F007
:10404000CBFC002001F0C8FCF32001F0C5FC0020EF
:1040500001F0C2FCE62001F0CBFC112001F0BCFC19
:10406000002001F0B9FC342001F0B6FC002001F082
:10407000B3FC562001F0B0FC002001F0ADFC76202E
:1040800001F0AAFC002001F0A7FC772001F0A4FCBD
:10409000002001F0A1FC662001F09EFC002001F050
:1040A0009BFC882001F098FC002001F095FC9920F1
:1040B00001F092FC002001F08FFCBB2001F08CFC91
:1040C000002001F089FC992001F086FC002001F01D
:1040D00083FC662001F080FC002001F07DFC55206F
:1040E00001F07AFC002001F077FC552001F074FC0F
:1040F000002001F071FC452001F06EFC002001F071
:104100006BFC432001F068FC002001F065FC4420BA
:1041100001F062FC002001F05FFCE72001F068FC88
:10412000322001F059FC002001F056FC552001F02E
:1041300053FC002001F050FC762001F04DFC0020E3
:1041400001F04AFC662001F047FC002001F044FC2D
:10415000672001F041FC002001F03EFC672001F0E7
:104160003BFC002001F038FC872001F035FC0020EA
:1041700001F032FC992001F02FFC002001F02CFC12
:10418000BB2001F029FC002001F026FC992001F061
:1041900023FC002001F020FC772001F01DFC002012
:1041A00001F01AFC442001F017FC002001F014FC7F
:1041B000562001F011FC002001F00EFC232001F03C
:1041C0000BFC002001F008FC332001F005FC00206E
:1041D00001F002FC452001F0FFFB002001F0FCFB98
:1041E000E82001F005FC002001F0F6FB002001F0C2
:1041F000F3FB992001F0F0FB002001F0EDFB87209C
:1042000001F0EAFB002001F0E7FB882001F0E4FB6D
:10421000002001F0E1FB772001F0DEFB002001F03F
:10422000DBFB662001F0D8FB002001F0D5FB8820E5
:1042300001F0D2FB002001F0CFFBAA2001F0CCFB63
:10424000002001F0C9FBBB2001F0C6FB002001F0FB
:10425000C3FB992001F0C0FB002001F0BDFB6620EC
:1042600001F0BAFB002001F0B7FB552001F0B4FBD0
:10427000002001F0B1FB552001F0AEFB002001F061
:10428000ABFB442001F0A8FB002001F0A5FB44207B
:1042900001F0A2FB002001F09FFB552001F09CFBE8
:1042A000002001F099FBE92001F0A2FBAA2001F017
:1042B00093FB002001F090FB002001F08DFB00201B
:1042C00001F08AFB002001F093FBAA2001F084FB9F
:1042D000CF2001F08DFB002001F07EFB002001F0DB
:1042E0007BFB002001F078FB002001F075FB002033
:1042F00001F072FB002001F06FFB002001F06CFB6D
:10430000002001F069FB002001F066FB002001F0B5
:1043100063FB002001F060FB002001F05DFB00204A
:1043200001F05AFB002001F057FB002001F054FB84
:10433000002001F051FB002001F04EFBF02001F0C5
:1043400057FB002001F048FB502001F045FB002006
:1043500001F042FB002001F03FFB002001F03CFB9C
:10436000F32001F045FB002001F036FBF92001F0BD
:104370003FFB062001F030FB102001F02DFB29202F
:1043800001F02AFB002001F027FB3A2001F030FB6E
:10439000552001F021FB112001F02AFB642003F0DD
:1043A000A5F9292001F024FB352001F021FB002094
:1043B00001F012FB512001F01BFBFF2001F00CFB70
:1043C000532001F015FB2C2001F006FB552001F0D5
:1043D0000FFB822001F000FB2C20FDE3A0427DD1E9
:1043E0004FF470435521184601F018FB4FF2010BB2
:1043F000AA21584601F012FB52214FF2020001F0AF
:104400000DFB08214FF2030001F008FB01214FF2E0
:10441000040001F003FB0D214FF4304001F0FEFADF
:104420000D214BF2010001F0F9FA0D214BF20200CF
:1044300001F0F4FA34214FF4364001F0EFFA342160
:104440004BF2016001F0EAFA34214BF2026001F014
:10445000E5FA0D214FF4314001F0E0FA0D214BF265
:10446000011001F0DBFA0D214BF2021001F0D6FA37
:1044700034214FF4374001F0D1FA34214BF201706E
:1044800001F0CCFA34214BF2027001F0C7FA00219E
:104490004FF4324001F0C2FA00214BF2012001F04A
:1044A000BDFA00214BF2022001F0B8FA24214FF4AA
:1044B000384001F0B3FA24214BF6010001F0AEFAC6
:1044C00024214BF6020001F0A9FA01214FF43F40EC
:1044D00001F0A4FA0F214FF4334000E0FEE301F0B5
:1044E0009DFA0F214BF2013001F098FA0F214BF2A7
:1044F000023001F093FA34214FF4394001F08EFA82
:1045000034214BF6011001F089FA34214BF60210E8
:1045100001F084FA08214FF4354001F07FFA0821B8
:104520004BF2015001F07AFA08214BF2025001F0EF
:1045300075FA03214FF4424001F070FA24214FF440
:104540003A4001F06BFA24214BF6012001F066FAA3
:1045500024214BF6022001F061FA00214FF43C4087
:1045600001F05CFA78214BF6014001F057FA002186
:104570004BF6024001F052FA00214FF43D4001F0A9
:104580004DFA78214BF6015001F048FA00214BF624
:10459000025001F043FA00214FF43E4001F03EFA90
:1045A00064214BF6016001F039FA00214FF45140CB
:1045B00001F034FA33214DF2011001F02FFA0021FD
:1045C0004DF2021001F02AFA34214DF2031001F0ED
:1045D00025FA00214DF2041001F020FA3A214DF2A3
:1045E000051001F01BFA00214DF2061001F016FA39
:1045F0004A214DF2071001F011FA00214DF2081086
:1046000001F00CFA5C214DF2091001F007FA0021CB
:104610004DF20A1001F002FA81214DF20B1001F067
:10462000FDF900214DF20C1001F0F8F9A6214DF230
:104630000D1001F0F3F900214DF20E1001F0EEF92A
:10464000E5214DF20F1001F0E9F901214DF21010B2
:1046500001F0E4F913214DF2111001F0DFF901210D
:104660004DF2121001F0DAF954214DF2131001F05D
:10467000D5F901214DF2141001F0D0F982214DF24B
:10468000151001F0CBF901214DF2161001F0C6F919
:10469000CA214DF2171001F0C1F902214DF2181094
:1046A00001F0BCF900214DF2191001F0B7F9022117
:1046B0004DF21A1001F0B2F901214DF21B1001F078
:1046C000ADF902214DF21C1001F0A8F934214DF290
:1046D0001D1001F0A3F902214DF21E1001F09EF908
:1046E00067214DF21F1001F099F902214DF22010BF
:1046F00001F094F984214DF2211001F08FF902218B
:104700004DF2221001F08AF9A4214DF2231001F09C
:1047100085F902214DF2241001F080F9B7214DF204
:10472000251001F07BF902214DF2261001F076F9F7
:10473000CF214DF2271001F071F902214DF228101E
:1047400001F06CF9DE214DF2291001F067F9022128
:104750004DF22A1001F062F9F2214DF22B1001F016
:104760005DF902214DF22C1001F058F9FE214DF2B5
:104770002D1001F053F903214DF22E1001F04EF9E6
:1047800010214DF22F1001F049F903214DF23010A4
:1047900001F044F933214DF2311001F03FF90321CA
:1047A0004DF2321001F03AF96D214DF2331001F063
:1047B00035F900214FF4524001F030F933214DF228
:1047C000012001F02BF900214DF2022001F026F921
:1047D00034214DF2032001F021F900214DF2042093
:1047E00001F01CF93A214DF2052001F017F90021E2
:1047F0004DF2062001F012F94A214DF2072001F096
:104800000DF900214DF2082001F008F95C214DF26C
:10481000092001F003F900214DF20A2001F0FEF811
:1048200081214DF20B2001F0F9F800214DF20C200E
:1048300001F0F4F8A6214DF20D2001F0EFF800216F
:104840004DF20E2001F0EAF8E5214DF20F2001F0C3
:10485000E5F801214DF2102001F0E0F813214DF2AE
:10486000112001F0DBF801214DF2122001F0D6F801
:1048700054214DF2132001F0D1F801214DF2142002
:1048800001F0CCF882214DF2152001F0C7F801218A
:104890004DF2162001F0C2F8CA214DF2172001F0A6
:1048A000BDF802214DF2182001F0B8F800214DF2B8
:1048B000192001F0B3F802214DF21A2001F0AEF8F0
:1048C00001214DF21B2001F0A9F802214DF21C201C
:1048D00001F0A4F834214DF21D2001F09FF80221CF
:1048E0004DF21E2001F09AF867214DF21F2001F0D1
:1048F00095F802214DF2202001F090F884214DF22C
:10490000212001F08BF802214DF2222001F086F8DF
:10491000A4214DF2232001F081F802214DF2242040
:1049200001F07CF8B7214DF2252001F077F8022143
:104930004DF2262001F072F8CF214DF2272001F030
:104940006DF802214DF2282001F068F8DE214DF2C9
:10495000292001F063F802214DF22A2001F05EF8CF
:10496000F2214DF22B2001F059F802214DF22C20BA
:1049700001F054F8FE214DF22D2001F04FF80321F3
:104980004DF22E2001F04AF810214DF22F2001F0B7
:1049900045F803214DF2302001F040F833214DF26B
:1049A000312001F03BF803214DF2322001F036F8BE
:1049B0006D214DF2332001F031F800214FF45340C6
:1049C00001F02CF833214DF2013001F027F80021DD
:1049D0004DF2023001F022F834214DF2033001F0A3
:1049E0001DF800214DF2043001F018F83A214DF283
:1049F000053001F013F800214DF2063001F00EF8F9
:104A00004A214DF2073001F009F800214DF208303B
:104A100001F004F85C214DF2093000F0FFFF0021A5
:104A20004DF20A3000F0FAFF81214DF20B3000F018
:104A3000F5FF00214DF20C3000F0F0FFA6214DF201
:104A40000D3000F0EBFF00214DF20E3000F0E6FFDC
:104A5000E5214DF20F3000F0E1FF01214DF2103061
:104A600000F0DCFF13214DF2113000F0D7FF0121DF
:104A70004DF2123000F0D2FF54214DF2133000F00D
:104A8000CDFF01214DF2143000F0C8FF82214DF21C
:104A9000153000F0C3FF01214DF2163000F0BEFFCB
:104AA000CA214DF2173000F0B9FF02214DF2183043
:104AB00000F0B4FF00214DF2193000F0AFFF0221E9
:104AC0004DF21A3000F0AAFF01214DF21B3000F028
:104AD000A5FF02214DF21C3000F0A0FF34214DF261
:104AE0001D3000F09BFF02214DF21E3000F096FFBA
:104AF00067214DF21F3000F091FF02214DF220306E
:104B000000F08CFF84214DF2213000F087FF02215C
:104B10004DF2223000F082FFA4214DF2233000F04C
:104B20007DFF02214DF2243000F078FFB7214DF2D5
:104B3000253000F073FF02214DF2263000F06EFFA9
:104B4000CF214DF2273000F069FF02214DF22830CD
:104B500000F064FFDE214DF2293000F05FFF0221FA
:104B60004DF22A3000F05AFFF2214DF22B3000F0C6
:104B700055FF02214DF22C3000F050FFFE214DF286
:104B80002D3000F04BFF03214DF22E3000F046FF98
:104B900010214DF22F3000F041FF03214DF2303053
:104BA00000F03CFF33214DF2313000F037FF03219C
:104BB0004DF2323000F032FF6D214DF2333000F013
:104BC0002DFF00214FF4544000F028FF33214DF217
:104BD000014000F023FF00E082E300214DF202409B
:104BE00000F01CFF34214DF2034000F017FF0021BC
:104BF0004DF2044000F012FF3A214DF2054000F062
:104C00000DFF00214DF2064000F008FF4A214DF251
:104C1000074000F003FF00214DF2084000F0FEFEC7
:104C20005C214DF2094000F0F9FE00214DF20A40EE
:104C300000F0F4FE81214DF20B4000F0EFFE002168
:104C40004DF20C4000F0EAFEA6214DF20D4000F0BE
:104C5000E5FE00214DF20E4000F0E0FEE5214DF2B0
:104C60000F4000F0DBFE01214DF2104000F0D6FEB7
:104C700013214DF2114000F0D1FE01214DF21240FE
:104C800000F0CCFE54214DF2134000F0C7FE01218C
:104C90004DF2144000F0C2FE82214DF2154000F0AA
:104CA000BDFE01214DF2164000F0B8FECA214DF2C2
:104CB000174000F0B3FE02214DF2184000F0AEFEA6
:104CC00000214DF2194000F0A9FE02214DF21A40D8
:104CD00000F0A4FE01214DF21B4000E003E300F0D0
:104CE0009DFE02214DF21C4000F098FE34214DF251
:104CF0001D4000F093FE02214DF21E4000F08EFE9A
:104D000067214DF21F4000F089FE02214DF2204044
:104D100000F084FE84214DF2214000F07FFE02214C
:104D20004DF2224000F07AFEA4214DF2234000F023
:104D300075FE02214DF2244000F070FEB7214DF2C5
:104D4000254000F06BFE02214DF2264000F066FE89
:104D5000CF214DF2274000F061FE02214DF22840A4
:104D600000F05CFEDE214DF2294000F057FE0221EA
:104D70004DF22A4000F052FEF2214DF22B4000F09D
:104D80004DFE02214DF22C4000F048FEFE214DF276
:104D90002D4000F043FE03214DF22E4000F03EFE78
:104DA00010214DF22F4000F039FE03214DF230402A
:104DB00000F034FE33214DF2314000F02FFE03218C
:104DC0004DF2324000F02AFE6D214DF2334000F0EA
:104DD00025FE00214FF4554000F020FE33214DF216
:104DE000015000F01BFE00214DF2025000F016FEB3
:104DF00034214DF2035000F011FE00214DF2045019
:104E000000F00CFE3A214DF2055000F007FE0021A3
:104E10004DF2065000F002FE4A214DF2075000F01C
:104E2000FDFD00214DF2085000F0F8FD5C214DF22F
:104E3000095000F0F3FD00214DF20A5000F0EEFDA4
:104E400081214DF20B5000F0E9FD00214DF20C5094
:104E500000F0E4FDA6214DF20D5000F0DFFD002131
:104E60004DF20E5000F0DAFDE5214DF20F5000F04A
:104E7000D5FD01214DF2105000F0D0FD13214DF26F
:104E8000115000F0CBFD01214DF2125000F0C6FD93
:104E900054214DF2135000F0C1FD01214DF2145088
:104EA00000F0BCFD82214DF2155000F0B7FD01214C
:104EB0004DF2165000F0B2FDCA214DF2175000F02D
:104EC000ADFD02214DF2185000F0A8FD00214DF279
:104ED000195000F0A3FD02214DF21A5000F09EFD82
:104EE00001214DF21B5000F099FD02214DF21C50A2
:104EF00000F094FD34214DF21D5000F08FFD022191
:104F00004DF21E5000F08AFD67214DF21F5000F057
:104F100085FD02214DF2205000F080FD84214DF2EC
:104F2000215000F07BFD02214DF2225000F076FD71
:104F3000A4214DF2235000F071FD02214DF22450C6
:104F400000F06CFDB7214DF2255000F067FD022105
:104F50004DF2265000F062FDCF214DF2275000F0B7
:104F60005DFD02214DF2285000F058FDDE214DF28A
:104F7000295000F053FD02214DF22A5000F04EFD61
:104F8000F2214DF22B5000F049FD02214DF22C5040
:104F900000F044FDFE214DF22D5000F03FFD0321B5
:104FA0004DF22E5000F03AFD10214DF22F5000F03E
:104FB00035FD03214DF2305000F030FD33214DF22C
:104FC000315000F02BFD03214DF2325000F026FD50
:104FD0006D214DF2335000F021FD00214FF4564079
:104FE00000F01CFD33214DF2016000F017FD00219F
:104FF0004DF2026000F012FD34214DF2036000F02A
:105000000DFD00214DF2046000F008FD3A214DF243
:10501000056000F003FD00214DF2066000F0FEFC8B
:105020004A214DF2076000F0F9FC00214DF20860C2
:1050300000F0F4FC5C214DF2096000F0EFFC00216F
:105040004DF20A6000F0EAFC81214DF20B6000F0A5
:10505000E5FC00214DF20C6000F0E0FCA6214DF2D1
:105060000D6000F0DBFC00214DF20E6000F0D6FC7C
:10507000E5214DF20F6000F0D1FC01214DF21060EE
:1050800000F0CCFC13214DF2116000F0C7FC0121AF
:105090004DF2126000F0C2FC54214DF2136000F09A
:1050A000BDFC01214DF2146000F0B8FC82214DF2EC
:1050B000156000F0B3FC01214DF2166000F0AEFC6B
:1050C000CA214DF2176000F0A9FC02214DF21860D0
:1050D00000F0A4FC00214DF2196000F09FFC0221B9
:1050E0004DF21A6000F09AFC01214DF21B6000F0B5
:1050F00095FC02214DF21C6000F090FC34214DF231
:105100001D6000F08BFC02214DF21E6000F086FC59
:1051100067214DF21F6000F081FC02214DF22060FA
:1051200000F07CFC84214DF2216000F077FC02212C
:105130004DF2226000F072FCA4214DF2236000F0D9
:105140006DFC02214DF2246000F068FCB7214DF2A5
:10515000256000F063FC02214DF2266000F05EFC49
:10516000CF214DF2276000F059FC02214DF228605A
:1051700000F054FCDE214DF2296000F04FFC0221CA
:105180004DF22A6000F04AFCF2214DF22B6000F053
:1051900045FC02214DF22C6000F040FCFE214DF256
:1051A0002D6000F03BFC03214DF22E6000F036FC38
:1051B00010214DF22F6000F031FC03214DF23060E0
:1051C00000F02CFC33214DF2316000F027FC03216C
:1051D0004DF2326000F022FC6D214DF2336000F0A0
:1051E0001DFC5521184600F019FCAA21584600F074
:1051F00015FC52214FF2020000F010FC08214FF282
:10520000030000F00BFC00214FF2040000F006FC4C
:10521000CC214FF4314000F001FC00214BF2011091
:1052200000F0FCFB05214FF4364000F0F7FB702145
:105230004FF4374000F0F2FB70214BF2017000F0A8
:10524000EDFB01214FF4384000F0E8FB03214BF661
:10525000010000F0E3FB03214BF6020000F0DEFB4F
:1052600003214BF6030000F0D9FB02214FF43C4030
:1052700000F0D4FB00214BF6014000F0CFFB0021F1
:105280004BF6024000F0CAFBD0214FF4494000F039
:10529000C5FB02214CF6011000F0C0FB50214CF67A
:1052A000021000F0BBFB50214CF6031000F0B6FBDF
:1052B00050214CF6041000F0B1FB00214FF4545083
:1052C00000F0ACFB55214FF4685000F0A7FB4FF401
:1052D000885000F08DFB782002F016FA4FF424502D
:1052E00000F086FBB9E0B842FCD1E22000F080FB80
:1052F0001D2000F071FB022000F06EFB042000F086
:105300006BFB642002F000FAE02000F071FB01204A
:1053100000F062FB0A2002F0E9F9E02000F068FBEF
:10532000032000F059FB0C2002F0E0F9012000F00E
:105330005FFB0A2002F0DAF9E62000F059FB2F208B
:1053400000F04AFBFF2000F047FBFF2000F044FB89
:10535000B02000F04DFB202000F03EFB002000F0CC
:105360003BFB032000F038FB40F21F3000F034FB21
:10537000012000F031FB40F2DF1000F02DFB002097
:1053800000F02AFBB42000F033FB042000F024FBE3
:1053900040F21F4000F020FB002000F01DFB2E20FB
:1053A00000F01AFB002000F017FB002000F014FBB7
:1053B000002000F011FB002000F00EFBB62000F0F2
:1053C00017FB022000F008FB4FF4037000F004FB11
:1053D000002000F001FB172000F0FEFA152000F07D
:1053E000FBFA002000F0F8FA002000F0F5FAF020B7
:1053F00000F0FEFA032000F0EFFA292000F0F8FA9E
:10540000D02000F0F5FA002000F0E6FABE2000F00F
:10541000EFFA052000F0E0FAFE2000F0DDFA0120AE
:1054200000F0DAFA002000F0D7FA002000F0D4FAF9
:10543000002000F0D1FAB82000F0DAFA032000F0E2
:10544000CBFA012000F0C8FABA2000F0D1FA01200E
:1054500000F0C2FA642000F063F8A888484505D03F
:10546000B04203D0A04201D0B84209D1052000903B
:1054700002906946D8F82C30D8E90102FBF7EEFA21
:10548000A98808A0FBF700F80020FDF749FD0848AF
:1054900001222021FBF797FD5046FDF71DFD15B0B9
:1054A000BDE8F08F4C43442049443A25780D0A006A
:1054B000000402581FB5FBF74BFF032201218DF8B2
:1054C0000010500701901B208DF8080000208DF877
:1054D0000C008DF809008DF80D008DF80A008DF88C
:1054E0000E0068468DF801208DF80B208DF80F1006
:1054F000FBF704FF0420FBF739FF1FBD0346012023
:1055000000E05843491EC9B2FBD27047034808B5B2
:105510000088ADF80000BDF8000008BD000008607C
:105520000246BE2000B500F063FA052000F054FAF0
:1055300000EE102A9FED0D1BB8EE400B20EE010B84
:10554000BCEEC00B10EE100A80B200F045FA01204C
:1055500000F042FAFF2000F03FFA002000F03CFA91
:105560005DF804EB002000F037BA0000666666665E
:1055700066660440F0B56C4D002341F6631429467D
:10558000AA798988012A01D01AB11BE0A14202D16F
:1055900018E0A14216D1082814D2DFE800F0040672
:1055A000080A0C0E101206200CE007200AE0042066
:1055B00008E0052006E0012004E0002002E00320CE
:1055C00000E0022045F21032A1F5134745F21056D3
:1055D000413F05D0914203D0B14201D0A14277D1E1
:1055E000082812D2DFE800F0110406080A0C0E1099
:1055F00080230AE0402308E0C02306E0202304E0E3
:10560000602302E0A02300E0E023B14202D14FF486
:10561000585000E03620914205D0B14203D0A1425B
:1056200001D043F00803194600F0F8F9AA88A24215
:105630000AD069889806288802D5884202D303E0F8
:10564000884201D929806880B242688941D100F03E
:10565000CFF9002000F0C0F96889401C80B200F04A
:10566000C7F9002000F0B8F96889801C80B200F00A
:10567000BFF92888401EC0F30F2000F0ADF96889FB
:10568000C01C80B200F0B4F92878401EC0B200F00F
:10569000A3F9A88900F0ACF9002000F09DF9A889D1
:1056A000401C80B200F0A4F9002000F095F9A88910
:1056B000801C80B200F09CF96888401EC0F30F2067
:1056C00000F08AF9A889C01C80B200F091F922E0AC
:1056D00028E000F08DF9002000F07EF9002000F0B5
:1056E0007BF92888401EC0F30F2000F075F9287858
:1056F000401EC0B200F070F9A88900F079F90020CE
:1057000000F06AF9002000F067F96888401EC0F3D5
:105710000F2000F061F9A878BDE8F040401EC0B24B
:1057200000F05AB9F0BD000010020024F0B53F4D62
:10573000060A0C4602462846270AA9884089A1F590
:105740001343413B28D0A1F5A643103B24D0A1F53B
:10575000C853633B2FD0A1F5AA43103B64D100F09E
:1057600047F9304600F038F96889401C80B200F0F3
:105770003FF9D0B200F030F9A88900F039F9384685
:1057800000F02AF9A889401C80B200F031F9E0B29B
:10579000BDE8F04000F020B900F02AF9304600F0F2
:1057A0001BF9D0B200F018F9A88900F021F93846A9
:1057B00000F012F9EBE7A97929B300F019F93046A6
:1057C00000F00AF9D0B200F007F92888401EC0F3B3
:1057D0000F2000F001F92878401EC0B200F0FCF85C
:1057E000A88900F005F9384600F0F6F8E0B200F0BC
:1057F000F3F86888401EC0F30F2000F0EDF8A87899
:10580000401EC0B2C4E72988891A491E8AB200F036
:10581000EFF8002000F0E0F8002000F0DDF8100ABA
:1058200000F0DAF8D0B2D9E7F0BD00001002002491
:105830002DE9F84F1F460E4682468B46580700D08A
:105840000120790800EBD700203A10FB01F0002579
:1058500002F0FF09C0B2009047E00C2F10D0102FCB
:1058600012D0182F14D0202F42D1224901EBC91099
:105870004FF00008445D200610D51F48026811E073
:105880001E4909EB490006E01D4901EB0910EFE74D
:105890001C4909EBC90001EB8000E9E70A9828B927
:1058A0001548426831465046FDF7B4FB6006761C49
:1058B000040E1548B6B24088B04219D9A6EB0B00C9
:1058C000B84209D10AF101005E461FFA80FA0E487B
:1058D000018851450CD906E008F1010000F0FF08ED
:1058E000B8F1080FC7D36D1CEDB200988542B4D350
:1058F000BDE8F88FC293000824000024027C000851
:105900007680000866860008100200242DE9FF4F0B
:1059100081B01D460027924680463C46DDF838B0EF
:10592000B9464FEA5B0627E0281B401EC1B20A2099
:10593000FFF7E4FDBAFBF0F00A21B0FBF1F201FB46
:10594000120027B9691E8C4201DA48B101275B4673
:105950003030CDF80090C2B206FB048080B206E081
:1059600006FB048020225B4680B2CDF800900299AD
:10597000FFF75EFF641CE4B2AC42D5D305B0BDE8CE
:10598000F08F2DE9F84F00F0FF08044610190D467E
:105990001FFA80FA4FF0000B58191FFA80F9DDE961
:1059A0000A7611E0544502D3E819444685B24D45C4
:1059B0000FD23B4629462046CDF800B0FFF738FF0E
:1059C00004EB570084B2761C3278A2F120005E28E6
:1059D000E8D9BDE8F88F000001B5BDF80000ADF8CA
:1059E0000000BDF800000149088008BD0000086003
:1059F00001B5BDF80000ADF80000BDF80000014998
:105A0000088008BDFEFF076002480349008908803E
:105A10007047000010020024FEFF0760024A108059
:105A2000901C018070470000FEFF0760104810B511
:105A300086B0016841F002010160006801210D4C4F
:105A400000F0020005900320CDE90001CDE902102D
:105A500069462046FBF7BAF9012220461146FBF7BA
:105A6000B2FA012220460221FBF7ADFA06B010BDC2
:105A7000E04402580004025808B500900548018B24
:105A8000C08A491E8BB2401E82B20021084600F037
:105A900049F808BDFC02002400B5AFB04FF0005338
:105AA0000093CDE9090102200B90CDE90C02684674
:105AB000FBF7DAFD002800D001202FB000BD000068
:105AC000084B10B51C465875A1888AB2218889B246
:105AD00020B1012801D1D9821A8310BDDA8219833D
:105AE00010BD0000FC020024F0B50C4F94B2DFF8AA
:105AF00030C03D467E7D2B68EA692D7D5CF82550DF
:105B000026B103FB01004243AC52F0BD7E68301A5F
:105B1000401E03FB001050432C52F0BDFC02002439
:105B20002C0000242DE9F043254E0024DDF81C90C4
:105B3000757D0DB1054606E077680D46B91A1A461F
:105B40003B1A491E5B1E3068521B96F814C0DFF8E2
:105B50007480871A00FB0150F6697F1E58F82CC02C
:105B6000BFB206FB00C51848066846F4000606608A
:105B700016484FF4403606600226466307640668FE
:105B800026F001060660C563591A4FF48033491C9C
:105B900003EB024211434164C0F83890016841F0C0
:105BA00001010160420202E0641C944202D2416899
:105BB0008907F9D5816841F002018160BDE8F08371
:105BC000FC0200242C000024D8440258001000528B
:105BD0002DE9FF5F00F0BEF9B84D01230827044608
:105BE0000626A0F5864042384FF4F0723AD0A4F56C
:105BF000E0404FF0170A84384FF4487140D003203A
:105C00004FF08C09A4F5E04CBCF1160C4FF4806BFE
:105C10004FF4167E42D0A4F5E048B8F118084FF4CE
:105C2000A06C47D0A4F50048B8F1160845D0A4F5FB
:105C30008058B8F1180843D04AF2010844454FF49F
:105C4000407949D140F25651C5E900198F21298187
:105C500046212982D521A98168811821E9811C2248
:105C60006882ADE04FF48870C5E900202B812820C0
:105C70006B81A8810520EF81582228826F829FE0E6
:105C8000C5E900122B812E206B81A881D220A5F8B6
:105C90000EA0288216201822688291E0C5E900BE75
:105CA000142129816881A020A5F80C90E98128821F
:105CB0000C2055E0C5E900C186E0C5E900BE83E0DF
:105CC000C5E900C1A5F80C900A212982102229817A
:105CD000E9816982688173E0A4F52048B8F102087F
:105CE00016D0A4F52048B8F103081FD0A4F5204C25
:105CF000BCF1040C29D0A4F52040053833D0A4F51C
:105D0000204006383ED0A4F52040073849D05BE05B
:105D1000C5E900C120212981302129825021A98192
:105D20006E810E21E9811622688249E0C5E900C929
:105D3000202129815021A9813021298207216981CF
:105D40000C21E981172268823AE0C5E900B988216F
:105D5000298118212982A021A9816E811D21E98133
:105D6000122268822CE04FF45470C5E900027020C2
:105D70002881A881102028822F226F81A5F80EA0EB
:105D80006E821DE0C5E9001E802028815820A88170
:105D90002820288204206881A5F80EA028226B8282
:105DA0000EE04FF42070C5E90002602028812F82A8
:105DB0003820A881022068812921E9813E22688259
:105DC000A0210520FFF768FE3D484FF000082A6833
:105DD0003D4F3E4B0280696841800220E8613948AE
:105DE00038603648A838C0E90038C0F80880A4F503
:105DF0008053C0F80C80183BC0F8108002D14FF0DF
:105E0000805303612C89631E43616B89A3F1010CEC
:105E1000C0F818C0B5F80CC06444A4F1010CC0F877
:105E20001CC0B5F80EC06344A3F1010CC0F820C03B
:105E3000A2F1010CA444C0F824C0A1F1010C9C44BF
:105E4000C0F828C0B5F810C062442244521EC26295
:105E50006A8A11441944491E016380F8368080F82B
:105E6000358080F834801548A838FBF717F90720EB
:105E7000CDE90086CDE902083968FF23022200201F
:105E800000F028F8A8880022114680B200902888E7
:105E900083B2104600F04CF80020FFF711FE0C48CA
:105EA0000122202185F81480FBF78DF804B04FF013
:105EB000FF30BDE8F05FFFF7DFBD0000FC0200240B
:105EC00010020024000000C02C000024001000502C
:105ED000000402582DE9F0438DB0164614AA134D64
:105EE00000240DF1240E92E88013009402942A6895
:105EF00001926D68CDE904634FEA08230395CDE96B
:105F000006734FEA092308938EE8260002460748E5
:105F10008DF8324069468DF83140A8388DF830C090
:105F2000FBF792F80DB0BDE8F0830000FC020024FE
:105F300070B51E46044603460548049DFBF78AF9E2
:105F400023462A4631460248BDE87040FBF7ACB90B
:105F5000540200242B4830B587B0016841F4007129
:105F60000160016801F400710591016841F48061EC
:105F7000016000686946244C00F480600590402070
:105F8000009000200190032003902046FAF71EFFA6
:105F90001E4D4420694600902846FAF717FF40211D
:105FA0002046FBF707F8042104462846FBF702F8D1
:105FB00044EA400428464021FAF7FCFF44EA800006
:105FC00010F0FF000CD001280DD002280ED00328BD
:105FD0000FD0042810D0052811D0002007B030BD04
:105FE00044F24230FAE747F28400F7E747F216003E
:105FF000F4E747F21800F1E748F21600EEE741F245
:106000001800EBE7E0440258002402580028025828
:10601000F0B504688B88E568C5F30B452B441D0477
:10602000882303EBC213E65806F47046E650046872
:106030000F68E668C6F30B46761C3E442E43E650D6
:1060400003688C89DD68C5F30A052C4425048C247B
:1060500004EBC2141E5906F470461E5103688F6883
:10606000DE68C6F30A06761C3E442E431E510468C1
:10607000942303EBC213E55825F00705E5500568A6
:106080000C69EC5091F8313005681F0291F83230FC
:106090001C040B7E1E069C2303EBC21355F803C0A1
:1060A0004FF0000C45F803C091F8305034433D43A5
:1060B00025430468E5500468982303EBC213E558B0
:1060C00025F0FF05E55005684C69EC500468A023F5
:1060D00003EBC213E55840F20776B543E550D1E92A
:1060E00007452C430568EC500468AC2303EBC2134E
:1060F000E55844F803C005684C6AEC500B698BB353
:10610000012B32D0042B32D0022B30D0032B2ED0D7
:10611000072B2CD001230568B02404EBC2142E59A0
:1061200006F0E0262E51D1E90065AD1B0E8D5D43D2
:106130005E43ED1D45EA064305682B510468B42310
:1061400003EBC213E5586FF30A05E5500468C96A0A
:10615000E1500068842101EBC211425842F0010273
:106160004250F0BDFFE70423D5E70323D3E7022322
:10617000D1E770477047000054482DE9F041524C78
:1061800086B0016841F002010160016841F0200120
:1061900001604E480C38016841F4804101604020A4
:1061A0000090022001900320DFF824810025694639
:1061B0000A270497CDE902504046FAF707FE04206B
:1061C00069460926049600904046FAF7FFFD0496BA
:1061D000C020404E694600903046FAF7F7FD4FF474
:1061E00040706946049700903046FAF7EFFD374853
:1061F0006438016841F480410160016821F4804104
:1062000001603148203881688906FCD43249016038
:1062100032494160016841F00101016081688906ED
:10622000FCD44FF49C71416181688907FCD5C16839
:1062300041F00201C16081688906FCD44FF483718A
:10624000416181688907FCD5C16841F00201C160E4
:1062500081688906FCD4224941610561816849074A
:10626000FCD530212170016841F004010160816892
:106270008907FCD5C16841F00201C16081688906C7
:10628000FCD481688906FCD4C56116494161164871
:10629000016821F480310160134970310A6822F0ED
:1062A00001020A600A1D156082060F4B78331A60DE
:1062B0001B1D0E4A1A6005220A60016841F48031F4
:1062C000016006B0BDE8F08120500052E044025861
:1062D00000040258001402581003000101041600C3
:1062E000C0030003EBEF180F24ED00E02D000303C3
:1062F0002DE9F047DFF8E48004460F464FF000092F
:10630000D8F80000C043800709D0344D283D2868E4
:1063100020F080602860FAF75BFE064607E0012067
:10632000BDE8F087FAF754FE801B02284ED8286893
:106330000001F7D4D8F80010226821F47C3141EA3A
:106340000231C8F80010207A4FF4FE02A188400202
:10635000491EA0F5007080B2C1F308010843A1896D
:10636000491E02EA01410843217C1202491E02EA49
:10637000016108431949103108601848001D01687F
:10638000626921F0C001114301600168A26921F036
:106390002001114301606FB10168012F0ED041F45B
:1063A00000110160286840F080602860FAF710FE54
:1063B00004460DE0016841F40021F2E741F4801148
:1063C000EFE7FAF705FE001B022801D90320A7E733
:1063D00028680001F5D54846A2E700002844025885
:1063E0002DE9F047DFF8E48004460F464FF000093E
:1063F000D8F80000C043800709D0344D283D2868F4
:1064000020F080502860FAF7E3FD064607E00120FF
:10641000BDE8F087FAF7DCFD801B02284ED828681B
:106420008000F7D4D8F80010228821F07C7141EA6E
:106430000251C8F80010207A4FF4FE02A1884002F1
:10644000491EA0F5007080B2C1F308010843A1897C
:10645000491E02EA01410843217C1202491E02EA58
:10646000016108431949183108601848001D016886
:10647000626921F44061114301600168A26921F45D
:106480000071114301606FB10168012F0ED041F01E
:1064900080710160286840F080502860FAF798FD0C
:1064A00004460DE0016841F48001F2E741F4000187
:1064B000EFE7FAF78DFD001B022801D90320A7E7BB
:1064C00028688000F5D54846A2E700002844025815
:1064D0003CB500210C460091019100B10224134803
:1064E0004069800101D50E203CBD114D6946A88848
:1064F00080B2FAF7BDFB0028F6D10198400313D50E
:10650000A88801210204372000F01EF83720FAF78E
:10651000F3F90028E8D101212246062000F014F802
:106520000620FAF7E9F93CBD25203CBD0070005279
:1065300034000024034A51686FF30901014351609C
:106540007047000000700052044B9A6000F03F005A
:1065500040EA012040F48050D8607047007000523B
:1065600010B5094C606221F07E40A062E06A03F041
:10657000010120F0FF0040EA021040EA410040F033
:106580000100E06210BD00000070005215480122B9
:1065900000B5134987B0202301600021C0E9011232
:1065A0000822C0E90323402343615301C0E90631B7
:1065B000130203625302C0E9093106210220009050
:1065C000CDE90121CDE90310059069460690054803
:1065D000FCF79EF8034800F007F807B000BD000084
:1065E0004041005220020024002301221846114697
:1065F00010B500F021F84FF4FA7001F085F800238F
:1066000001221846022100F017F80023082218463C
:10661000032100F011F8012240F22223042100207E
:1066200000F00AF8BDE81040024840F2A521FCF74E
:1066300031B90000200200241FB5002410B1012848
:1066400002D002E0102400E008240748CDE902232C
:106650004FF6FF72CDE900146946FCF72CF90028CB
:1066600000D0012004B010BD200200240E4910B556
:10667000044600200978032906D019B1012901D068
:10668000022902D1022C01D3272010BDE0B2FFF76E
:106690001FFF0028F9D1054A516821F4404141EA21
:1066A000843189B2516010BD340000240070005262
:1066B0002DE9F04783494FF0000CDFF80CA24FF0B2
:1066C00001090B7880F856308988A0F85410DAF860
:1066D00000100A0E95090570C2F38305457002F09B
:1066E000030282700A0CC2700A0A02714171DAF860
:1066F0000420110E0C01C2F3074101F00F0844EA17
:106700001114C480C2F3072180F80880CC094472B8
:10671000C1F380148472C1F34014C472C1F3001435
:106720000473544680F80DC0A468260EC4F30745D0
:10673000C4F3072733B1012B04D0032B02D0022B63
:1067400030D03EE08907D2B2090D41EA820141EA28
:1067500096120261C6F3C201017506F00701417588
:1067600069098175C5F38201C175A9074B0F3946C7
:1067700043EAD1150576AD1C09FA05F3DE17521C64
:10678000A2FB03570CFB037302FB063309FA08F262
:106790000265A5FB026703FB027205FB0C22C0E940
:1067A00012620EE09106890A41EA062239462A431E
:1067B0000261521C530BD204C0E912234FF4007241
:1067C0000265C1F38012427689064A0EE1B242EABE
:1067D000D112827601F07F01C176DAF80C20110E19
:1067E000CB090377C1F341134377C1F382038907D0
:1067F00000F81E3F0B0FC2F3074143EA91134370A9
:10680000C1F34013837001F0010180F803C00171EE
:10681000C2F30721CB094371C1F380138371C1F324
:106820004013C371C1F300130372C1F381034372B8
:1068300001F003018172C2F34601234AC1724B4643
:10684000103280F80C9011680C0E84730C0CC1F39C
:10685000072545EA042404820C0651680D0E44EA1B
:106860000544C1F3074544EA0524C1F307252C4339
:10687000C0F81240817591680C0EC4750C0CC1F300
:1068800007252406C9B244EA054444EA0124D16834
:1068900044EA1164C0F81A40847FC1F3074244EA15
:1068A000121484771207C1F3072444EA12520284B7
:1068B000C1F3460180F8221080F823306046BDE81D
:1068C000F08700003400002420030024374810B56E
:1068D00086B0016841F480310160006800F48030C6
:1068E000059032480C30016841F0040101600168F4
:1068F00001F004010591016841F0080101600068A0
:106900000024694600F0080005904FF4F85000900C
:106910000220CDE90104032003900C2004902448B8
:10692000FAF754FA0420009022486946FAF74EFA22
:106930002148046044608460C46044628462C4622C
:106940001E498163C463002202213120FAF72EFD23
:106950003120FAF71EFD00F09BF8194C030014D10A
:1069600000F032F8030010D12046FFF7A1FE03002B
:106970000BD1B4F85400000400F02CFA030004D149
:106980000120FFF773FE030003D00E4800780328B0
:1069900007D194F8560038B1012805D00420FFF73C
:1069A000C9FD06B0184610BD0620F8E7D4440258C9
:1069B00000080258000C025800700052FF0FE01F40
:1069C000400300243400002438B52E4C0120ADF8DB
:1069D0000000206880071ED02B4D287804284ED058
:1069E000002203210220FFF7AFFDF9F7A7FF0028DF
:1069F00012D1616925480160A1694160E169816046
:106A0000216AC160287840B1012806D0062804D048
:106A1000022802D00CE0252038BD002201210320ED
:106A2000FFF792FD03206946F9F7C2FF0028F3D172
:106A3000287803280AD1BDF80000012102040320B0
:106A4000FFF782FDF9F77AFF0028E5D128780428BE
:106A500015D0BDF800000321686002040920FFF78B
:106A600073FDF9F76BFF0028D6D16169074810382C
:106A70000160A1694160E1698160216AC160002013
:106A800038BD0000007000523400002430030024A0
:106A90002DE9F04FDFF8F4A000273E463C463D4686
:106AA000B9465346CAF80470FA20FFF743FD0320A5
:106AB0001860002211461046FFF746FDF9F706FF61
:106AC00028B17F1CFFB24A2FF3D3BDE8F08F01211C
:106AD0004FF4D5720820FFF737FDF9F79DFFDFF877
:106AE000B0B020B901218BF800104FF0804900228E
:106AF00001213720FFF728FD3720F9F7FDFE4FF67B
:106B0000FF78D8B1234F5646A5B336E000220121C5
:106B10003720FFF719FD3720F9F7EEFE0028D4D112
:106B200001213A462920FFF70FFDF9F72BFF002836
:106B3000CBD1DAF81460F50F641C02E0164949EA7B
:106B400001070DB94445E1D3444518D216F0804FF2
:106B5000BBD002228BF80020B7E701213A46084655
:106B6000FFF7F2FCF9F70EFF0028AED17169CD0FE7
:106B7000641CC9E7FFE74445EFD3444501D31B201C
:106B8000A3E703218BF800109FE70000007000527C
:106B9000340000240080FF80000010802DE9F05FA9
:106BA000DFF874B10021DDE90A97164605464FF07B
:106BB000FF34CBF82C10DFF864A19AF8000002280B
:106BC00004D1560A4FF4007946EAC3564A460121D9
:106BD0001020FFF7B9FC1020F9F78EFE5FEA0008DD
:106BE00006D001464EA0F9F74FFC4046BDE8F09FA5
:106BF00007FB09F1012320460922FFF7B1FCDBF86E
:106C00000C10D84641F04001CBF80C10012F324651
:106C10004FF001010BD91220FFF796FC1220F9F773
:106C20006BFE06000BD043A0F9F72EFC71E011209B
:106C3000FFF78AFC1120F9F75FFE0600D6D1F9F7BD
:106C400084FB444910E0D8F8340000040AD5002041
:106C5000D8F8802045F82020401C0828F8D320359B
:106C60000C4601E0BCB1641ED8F8340010F4957FE6
:106C7000E9D0D8F80C0020F04000C8F80C00F9F773
:106C800066FBD8F83400000707D5D8F8380040F084
:106C90000800C8F838000420A8E7D8F834008007B6
:106CA00011D5D8F8380040F00200C8F83800012F9C
:106CB00007D9002201210C20FFF746FC0C20F9F730
:106CC0001BFE022092E7D8F83400800607D5D8F8DA
:106CD000380040F02000C8F83800062086E7D8F8D1
:106CE0003400C00512D5012F10D99AF8000018B150
:106CF000012801D0022809D1002201210C20FFF730
:106D000023FC0C20F9F7F8FD0600C5D11248C8F89D
:106D1000380030466AE7000000700052340000245A
:106D200053444D4D435F53656E645F436D643D2531
:106D3000640D0A0053445F434D445F524541445F34
:106D40004D554C545F424C4F434B204572726F720D
:106D50000D0A0000FFFF7F00FF0FE01F2DE9FC5F21
:106D60000D461A494FF0000807464046924606462F
:106D7000097809B1EE0D6D02BA074FF4007119D010
:106D800000248346894612E00120CDE9009060028C
:106D900042190F484BEB0603FFF700FF0C498046F2
:106DA0004A463846F9F718FC641C07F50077544545
:106DB000EAD307E0CDE9001A2A4633463846FFF702
:106DC000EDFE80464046BDE8FC9F000034000024F4
:106DD0009803002401210246072000B5FFF7B4FB09
:106DE0005DF804EB0720F9F787BD704770B5294CB3
:106DF0009CB0256825F004052560264C00260C343F
:106E0000256845F440452560256805F440451B95F7
:106E10002568AD04FCD5012400940CAD0396240430
:106E2000019402240994CDE90A410796082485E8D3
:106E30000D00CDE910466846FBF71CFA98B9FFF73C
:106E40009BF93F2013900320CDE914064020010157
:106E5000CDE91640CDE9180150201A90022113A85F
:106E6000FBF75AF810B101201CB070BD0A48016848
:106E700041F0800101600848F430016841F00201EE
:106E80000160006800F002001B90F9F797FF0020F6
:106E9000EAE700000C48025800440258FAF79EB88E
:106EA0001C48016841F4700101601B49086840F00A
:106EB00001000860184A0020103210600A68174B61
:106EC0001A400A60144A18321060121D1060121D18
:106ED0001060114A28321060121D1060121D1060DF
:106EE000121D1060121D1060121D1060121D106026
:106EF000121D10600A6822F480220A60064960317F
:106F0000086001200649C1F80801C006014980391E
:106F10000860704788ED00E0004402587FEDF6EA13
:106F20000080005190F83410C90706D001684A6803
:106F3000836B22F400321A434A6090F834108907B8
:106F400006D501684A68C36B22F480321A434A604E
:106F500090F83410490706D501684A68036C22F49A
:106F600080221A434A6090F83410090706D5016858
:106F70004A68436C22F400421A434A6090F8341085
:106F8000C90606D501688A68836C22F480521A43C8
:106F90008A6090F83410890606D501688A68C36C47
:106FA00022F400521A438A6090F83410490611D531
:106FB00001684A68036D22F480121A434A60016D29
:106FC000B1F5801F06D101684A68436D22F4C00202
:106FD0001A434A6090F83410090606D501684A68D9
:106FE000806D22F4002202434A607047F8B5002504
:106FF0000446C567F9F7ECFF0746206800686FF0A4
:107000007E46000708D500223B464FF4001120467B
:10701000009600F0FBFA60B92068006840070AD5C6
:1070200000223B464FF480012046009600F0EEFA25
:1070300008B10320F8BD202084F8790084F87A0094
:10704000002084F87850F8BD10B5806B0021A0F8BE
:107050006A10A0F86210FBF7D4FC10BD01680A6842
:1070600022F490720A6001688A6822F001028A6044
:10707000202180F87A10704710B5B0F86C2090F895
:107080007A300168222B05D0088B40F00800088375
:10709000022010BD898C8368B3F5805F01D103693C
:1070A0006BB11140426E531C43661170B0F86A1008
:1070B000491E0904090CA0F86A1007D015E0436EB8
:1070C00011401980416E891C4166EFE701680A682A
:1070D00022F490720A6001688A6822F001028A60D4
:1070E000202180F87A10FBF71DFE002010BD000063
:1070F0002DE9F04F044600688025FD4B0021D4F8AF
:1071000010C087B0A6680F46D4F81C8046EA0C066B
:10711000D4F814C0A26A4CEA080C46EA0C063243C2
:107120000668DFF8D0C306EA0C061643066020683E
:107130004268E66822F44052324342602268A06905
:107140009A4201D0266A3043A66AB6F1005F04D1A4
:10715000D4E90B6C46EA0C0630439668DFF898C316
:1071600006EA0C06064396602068C26A666A22F048
:107170000F023243C262E14E2068E14AB04210D1B0
:10718000126802F03802182A74D005DCCAB3082A43
:107190007AD0102A47D179E0202A7BD0282A7CD1C6
:1071A0007AE0D84EB04209D1126802F00702062AEE
:1071B00073D2DFE802F053696B6D6F71D24EB0424B
:1071C00009D1126802F00702062A66D2DFE802F04F
:1071D000465C5E606264CD4EB04209D1126802F036
:1071E0000702062A59D2DFE802F0394F51535557AA
:1071F000C74EB0420BD1126802F00702062A4CD2E9
:1072000000E00EE0DFE802F02A4042444648C14E6A
:10721000B04209D1126802F03802182A38D0BBDC1B
:10722000B4E74FF0010538E0BB4EB04209D1126817
:1072300002F00702062A30D2DFE802F01026282AE0
:107240002C2EB64EB0420BD1126802F00702062A6D
:1072500023D2DFE802F003191B1D1F2100251CE0CB
:1072600098421AD1A64A121D126802F00702062A95
:1072700013D202E00CE007E00CE0DFE802F00305C7
:1072800007090B0D022508E0042506E0402504E06F
:10729000082502E0102500E02025DFF864B2A04EAA
:1072A0009842DFF880A2ABF1540B73D1102D31D08E
:1072B00006DC022D09D0042D0AD0082D2FD111E0B3
:1072C000202D29D0402D2AD107E0FAF7BBF813E092
:1072D0006846FAF7CDF801980EE003A8FAF746F9E8
:1072E000049809E0DBF800105846890610D50068BC
:1072F000C0F3C1012AFA01F0002811D06168894663
:1073000001EB410181420AD8B0EB093F07D808E000
:107310005046F3E78448F1E74FF40040EEE70127D9
:1073200033E1102D4FF000084ED006DC022D0FD0B7
:10733000042D15D0082D04D12DE0202D4AD0402D4C
:1073400013D00127794AA0F54071914270D9E6E740
:10735000FAF778F8626A0023414636F812200DE009
:107360006846FAF785F8019803E003A8FAF7FEF8F3
:1073700004980023616A36F811201946F9F70CF8D1
:1073800062680902030241EA10615008181841EBD3
:10739000080115E032E0DBF800105846890609D5EF
:1073A00000680023C0F3C1012AFA01F0616A36F8CF
:1073B000112015E0606A002336F8102050460FE0D7
:1073C0000023F8F7E9FFBDE7606A002336F81020D4
:1073D000554805E0606A002336F810204FF400405D
:1073E0000021F8F7D9FF0902020241EA10614FEAD1
:1073F000590010184A4641EB0801E1E7E3694FF4F0
:10740000004293424DD1082D23D005DC8DB1012DD2
:1074100012D0042D06D112E0102D35D0202D3AD0F7
:10742000402D11D0012721F00F00C1F34201084384
:107430005AE0FAF777FE16E0FAF78AFE13E068469C
:10744000FAF716F801980EE003A8FAF78FF80498F7
:1074500009E0DBF800105846890608D50068C0F33B
:10746000C1012AFA01F0616A36F8111010E0606A71
:1074700036F81010BAFBF1F04100606801EB5001E2
:10748000B1FBF0F081B2CEE7606A36F81010264802
:10749000B0FBF1F0F0E7606A36F81000B2FBF0F0F4
:1074A000EAE7082D4AD00ADC0DB3012D43D0042DA4
:1074B0007FF44DAF6846F9F7DBFF019809E0102D26
:1074C00052D0202D55D0402DF2D103A8FAF74EF816
:1074D0000498616A36F81110B0FBF1F1606801EBB5
:1074E0005001B1FBF0F080B22168C8604DE01FE0B0
:1074F000000C0058F369FFCFFFF4FF1100100140AA
:10750000544402580044004000480040004C0040F1
:10751000005000400014014000780040007C004012
:10752000EA7B00080090D00300093D00FFFC0F003B
:10753000FAF7F8FDCDE7FAF70BFECAE7DBF8002013
:10754000594692060AD50968C1F3C1022AFA02F126
:10755000626A36F81220B1FBF2F20FE0616A36F887
:107560001120BAFBF2F209E0616A36F811200949EC
:10757000F1E7616A36F81110B2FBF1F2616802EBD3
:107580005102B2FBF1F189B2C16007B03846BDE8E3
:10759000F08F000000093D0090F87910212901D0FA
:1075A00002207047B0F8621021B18168B1F5805FA8
:1075B00013D014E001680A68920004D58A6822F4A6
:1075C00000028A6003E00A6822F080020A60006814
:1075D000016841F0400101600CE0016961B1C16DD9
:1075E0004A1CC265026809781185B0F86210491E0C
:1075F000A0F8621000207047C16D02680988C1F3CD
:1076000008011185C16D891CC165EEE72DE9F041C6
:107610001E46174688460446069D1CE0681C1AD084
:1076200025B1F9F7D5FC801BA84214D92068016860
:1076300021F4D07101602068816821F0010181602E
:10764000202084F8790084F87A00002084F87800FB
:107650000320BDE8F0812068C16938EA010004D048
:107660000020B842DAD00020F3E70120F9E700005B
:1076700070B50D4D00240D48FBF7CAF902E0641CFB
:10768000AC4204D80948FBF7BDF92028F7D1002403
:1076900002E0641CAC4206D8054901220348FBF70E
:1076A000EDFA0028F5D170BDFFFF01004401002470
:1076B0000C000024FEE70907090E002804DB00F196
:1076C000E02080F80014704700F00F0000F1E02087
:1076D00080F8141D7047704710B504460420FBF76E
:1076E0006FF90148046010BD0800002470B5002443
:1076F00005464FF47A7603E0304600F005F8641C46
:10770000AC42F9D370BD000070B54FF0E025002108
:107710006C69094AAB6912685043AA699A42FCD065
:1077200002D2A3EB020302E0A4EB020633441944A5
:1077300013468142F1D370BD080000240349CA6991
:107740005206FCD5C2B20A85704700000010014005
:107750001CB50024F9F776F8F9F748FC0423022257
:107760000521A020FFF742FB4FF4C870FFF7B4FFDC
:107770004FF4E13000F010FAFEF758F9FBF700FB88
:10778000FEF704FFFBF7C4FC002000F03FF95C4F5C
:107790004FF478401025C8222B463221386059A07A
:1077A000CDE900501E20FEF7ECF85BA01023C822A4
:1077B000CDE9005046211E20FEF7E3F85AA0102321
:1077C000C822CDE900505A211E20FEF7DAF85AA04F
:1077D0001023C822CDE900506E211E20FEF7D1F8FB
:1077E00058A01023C822CDE9005082211E20FEF7A8
:1077F000C8F8DFF864914FF4FA761BE057A0102325
:10780000C822CDE9005096211E20FEF7BAF8304676
:10781000FFF76CFF55A01023C822CDE90050962138
:107820001E20FEF7AEF83046FFF760FF0221484603
:10783000F9F7C5FBFFF74AF80028DFD100F020F97F
:107840001F2038604DA01023C822CDE9005096219A
:107850001E20FEF796F84DA01023C822CDE9005057
:10786000AA211E20FEF78DF84E4805230095D0E989
:1078700012100A0D42EA0032AA218620FEF746F8CD
:107880000020FBF7BDFA012809D101224046002162
:10789000FFF764FA01000FD043A0F8F7F5FD641C70
:1078A0000A20E4B2FFF722FF142CE9D10221484656
:1078B000F9F785FB0024E3E73EA01023C822CDE9B9
:1078C0000050BE211E20FEF75CF840A0F8F7DCFD5A
:1078D00000264FF4007742A018F80610F8F7D4FD00
:1078E000761CBE42F7D33FA0F8F7CEFD41A010238F
:1078F000C822CDE90050BE211E20FEF742F8CEE797
:1079000024000024504F4C41524953204837353011
:107910002F46373530000000534420434152442065
:10792000544553540000000041544F4D40414C49D0
:10793000454E54454B000000323031392F352F3140
:10794000300000004B4559303A5265616420536560
:1079500063746F72203000000004025853442043C7
:10796000617264204572726F72210000506C656113
:10797000736520436865636B2120000053442043F6
:10798000617264204F4B202020200000534420438C
:107990006172642053697A653A20202020204D428C
:1079A00000000000400300246572723A25640D0A4D
:1079B000000000005553415254312053656E6469F4
:1079C0006E6720446174612E2E2E0000534543548F
:1079D0004F52203020444154413A0D0A000000002B
:1079E000257820000D0A4441544120454E44454429
:1079F0000D0A00005553415254312053656E6420E6
:107A000044617461204F76657221000030B50446F0
:107A10000748084D002150F82400820005EB84003F
:107A2000006A00F027F80120291981F8380030BDDC
:107A300044C300083C0000240C4B002210B50C4C41
:107A4000114653F8203004EB800005E0046A54F836
:107A5000214004B1521C491C8B42F7D84FF47A7074
:107A60004243B2FBF3F080B210BD000044C30008F3
:107A70003C00002401E000F8011B521EFBD27047BD
:107A800010B5154C94F8560030B1012806D00228E4
:107A90001ED0032805D11DE010A000E015A0F8F7C6
:107AA000F3FC14F82C1F19A0F8F7EEFC218D1EA092
:107AB000F8F7EAFCD4E90710090D41EA00311EA0ED
:107AC000F8F7E2FC616A22A0BDE81040F8F7DCBCE0
:107AD00025A0E4E72AA0E2E74003002443617264A2
:107AE00020547970653A534453432056312E310D5A
:107AF0000A0000004361726420547970653A53446F
:107B000053432056322E300D0A0000004361726448
:107B1000204D616E75666163747572657249443A91
:107B200025640D0A00000000436172642052434145
:107B30003A25640D0A0000004361726420436170BD
:107B400061636974793A2564204D420D0A00000092
:107B50004361726420426C6F636B53697A653A25A6
:107B6000640D0A0D0A0000004361726420547970AC
:107B7000653A534448432056322E300D0A00000027
:107B80004361726420547970653A4D4D43204361DE
:107B900072640D0A000000000B490A4A10B5C1E9E1
:107BA000002000208860C860086188610C2048615E
:107BB0000846FAF7EDFFBDE81040044901220248EB
:107BC000FBF75CB800100140440100240C000024C5
:107BD0004FF04070E1EE100A704700000000010213
:107BE000030401020304060708090100020004005F
:107BF000060008000A000C00100020004000800071
:107C00000001000000000000000000000000000073
:107C100000003F4000000000000000003000400075
:107C200030004000000009000BC03D000BC03D00CB
:107C3000090018C024407FE0224031800000180075
:107C400024C01B000D803240018003801C4027406F
:107C50001C80074000401000600000000000000091
:107C600000000000000000001F80204040200000B5
:107C7000402020401F8000000000090006001F80F7
:107C8000060009000000040004003F800400040016
:107C90000000001000600000000000000000040070
:107CA0000400040004000400000000000040000084
:107CB000000000000000002001C006003800400065
:107CC00000001F802040204020401F800000000056
:107CD00010403FC000400000000018C0214022407A
:107CE00024401840000010802040244024401B8085
:107CF000000002000D0011003FC0014000003C8068
:107D0000244024402440238000001F80244024403D
:107D10003440038000003000200027C038002000DD
:107D200000001B802440244024401B8000001C00D5
:107D300022C0224022401F800000000000000840B6
:107D400000000000000000000000046000000000CF
:107D50000000000004000A001100208040400900DB
:107D600009000900090009000000000040402080CF
:107D700011000A000400180020002340240018000D
:107D800000001F802040274029401F400000004085
:107D900007C039000F0001C0004020403FC0244010
:107DA00024401B8000001F80204020402040308065
:107DB000000020403FC0204020401F8000002040A5
:107DC0003FC024402E4030C0000020403FC024402F
:107DD0002E00300000000F00108020402240338031
:107DE000020020403FC0040004003FC0204020406B
:107DF00020403FC020402040000000602020202084
:107E00003FC02000200020403FC024400B0030C075
:107E1000204020403FC020400040004000C03FC004
:107E20003C0003C03C003FC0000020403FC00C406D
:107E300023003FC020001F802040204020401F80A2
:107E4000000020403FC024402400180000001F8094
:107E50002140214020E01FA0000020403FC02440DE
:107E6000260019C0004018C0244024402240318020
:107E70000000300020403FC02040300000002000C3
:107E80003F80004000403F80200020003E0001C0B5
:107E9000070038002000380007C03C0007C0380049
:107EA0000000204039C0060039C0204000002000FA
:107EB000384007C0384020000000304021C0264034
:107EC000384020C00000000000007FE0402040203B
:107ED0000000000070000C00038000400000000063
:107EE000402040207FE00000000000002000400013
:107EF0002000000000000010001000100010001012
:107F00000010000000004000000000000000000021
:107F100002800540054003C0004020003FC00440EF
:107F20000440038000000000038004400440064039
:107F3000000000000380044024403FC000400000D7
:107F400003800540054003400000000004401FC0BE
:107F5000244024402000000002E005500550065057
:107F6000042020403FC00440040003C00040000043
:107F7000044027C000400000000000100010041062
:107F800027E00000000020403FC00140070004C07F
:107F90000440204020403FC000400040000007C097
:107FA000040007C0040003C00000044007C00440F0
:107FB000040003C00040000003800440044003802C
:107FC0000000041007F0045004400380000000008B
:107FD00003800440045007F00010044007C0024032
:107FE000040004000000000006400540054004C0F5
:107FF0000000000004001F80044000400000040056
:1080000007800040044007C000400400070004C08F
:10801000018006000400060001C0070001C0060040
:108020000000044006C0010006C004400000041027
:10803000071004E00180060004000000044005C0B1
:108040000640044000000000000004007BE04020E7
:108050000000000000000000FFF000000000000031
:1080600040207BE004000000000040008000400051
:108070002000200040000000000000000000000080
:108080000000000000000000000000001FCC000CF9
:108090000000000000000000080030006000080040
:1080A000300060000000022003FC1E20022003FCC0
:1080B0001E200220000000000E1811043FFF108453
:1080C0000C78000000000F0010840F3800C0077803
:1080D00018840078000000780F8410C411240E98D2
:1080E00000E4008400080800680070000000000040
:1080F00000000000000000000000000007E0181869
:10810000200440020000000040022004181807E08C
:108110000000000000000240024001800FF00180DA
:108120000240024000000080008000800FF80080C4
:108130000080008000000001000D000E0000000023
:10814000000000000000000000800080008000802F
:108150000080008000800000000C000C0000000087
:108160000000000000000000000600180060018010
:10817000060018002000000007F008081004100492
:10818000080807F000000000080408041FFC0004B1
:1081900000040000000000000E0C10141024104415
:1081A00011840E0C000000000C18100411041104BE
:1081B00012880C700000000000E003200424082452
:1081C0001FFC0024000000001F98108411041104FB
:1081D000108810700000000007F0088811041104D6
:1081E00018880070000000001C00100010FC130034
:1081F0001C001000000000000E3811441084108490
:1082000011440E38000000000700088C1044104490
:10821000088807F00000000000000000030C030CB9
:108220000000000000000000000000010106000046
:108230000000000000000000008001400220041047
:108240000808100400000220022002200220022060
:108250000220022000000000100408080410022080
:1082600001400080000000000E001200100C106C95
:1082700010800F00000003E00C1813E4142417C44E
:10828000082807D000000004003C03C41C4007403D
:1082900000E4001C000410041FFC1104110411046C
:1082A0000E880070000003E00C1810041004100485
:1082B00010081C10000010041FFC1004100410040F
:1082C000080807F0000010041FFC1104110417C473
:1082D00010040818000010041FFC1104110017C03E
:1082E00010000800000003E00C18100410041044F3
:1082F0001C780040000010041FFC108400800080E7
:1083000010841FFC10040000100410041FFC100453
:1083100010040000000000030001100110011FFE06
:1083200010001000000010041FFC110403801464EE
:10833000181C1004000010041FFC100400040004AA
:108340000004000C000010041FFC1F0000FC1F00B4
:108350001FFC1004000010041FFC0C04030000E0CC
:1083600010181FFC100007F0080810041004100477
:10837000080807F0000010041FFC10841080108013
:1083800010800F00000007F0081810241024101CA3
:10839000080A07F2000010041FFC1104110011C0AC
:1083A00011300E0C000400000E1C11041084108407
:1083B00010441C3800001800100010041FFC1004AA
:1083C00010001800000010001FF810040004000442
:1083D00010041FF8100010001E0011E0001C0070B7
:1083E00013801C0010001FC0103C00E01F0000E0C4
:1083F000103C1FC000001004180C163401C001C04E
:108400001634180C100410001C00130400FC130494
:108410001C00100000000804101C106410841304D9
:108420001C04101800000000000000007FFE400245
:10843000400240020000000030000C000380006099
:10844000001C0003000000004002400240027FFECA
:10845000000000000000000000002000400040007C
:1084600040002000000000010001000100010001A7
:108470000001000100010000400040002000000059
:1084800000000000000000000098012401440144A5
:10849000014400FC000410001FFC008801040104DA
:1084A00000880070000000000070008801040104D2
:1084B000010400880000000000700088010401042D
:1084C00011081FFC0004000000F8014401440144AD
:1084D000014400C800000000010401040FFC110465
:1084E000110411001800000000D6012901290129FA
:1084F00001C90106000010041FFC008401000100F6
:10850000010400FC000400000104190419FC00042B
:108510000004000000000000000300010101190137
:1085200019FE0000000010041FFC0024004001B4EC
:10853000010C010400000000100410041FFC0004E2
:10854000000400000000010401FC0104010001FC22
:108550000104010000FC010401FC00840100010091
:10856000010400FC0004000000F8010401040104FF
:10857000010400F80000010101FF0085010401046D
:1085800000880070000000000070008801040104F1
:10859000010501FF00010104010401FC0084010444
:1085A000010001800000000000CC0124012401240E
:1085B00001240198000000000100010007F80104F7
:1085C000010400000000010001F8000400040004A0
:1085D000010801FC0004010001800170000C001082
:1085E00001600180010001F0010C003001C0003089
:1085F000010C01F0010000000104018C0074017005
:10860000018C01040000010101810171000E0018BC
:1086100001600180010000000184010C013401446B
:108620000184010C000000000000000000000100B7
:108630003EFC400240020000000000000000FFFF7E
:108640000000000000000000400240023EFC01006B
:10865000000000000000000060008000800040007A
:10866000400020002000000000000000000000008A
:1086700000000000000000000000000000000000FA
:1086800000000000000000000000000000000000EA
:108690000000000000000000000F80380FFE380FBF
:1086A0008038000000000000000000000000000012
:1086B000000000000100000600000C00003800006F
:1086C0003100000600000C000038000030000000FF
:1086D00000000000000061800067F807F980006179
:1086E000800061800061800061800067F807F98088
:1086F00000618000000000000000000001C0E003F5
:10870000E0F00630080418081FFFFE040E08078773
:10871000F00381E000000000000001F000060C0002
:10872000040408060C7001F9C0000E00003BE000D4
:10873000EC18070808040C180003E0000000000112
:10874000E00007F003F818041C0804170807E1D03C
:1087500003C0E00023B0003C080020080000100027
:1087600000000000000100003100003200001C0089
:1087700000000000000000000000000000000000F9
:1087800000000000000000000000000000000000E9
:108790000000000000007F0001FFC00780F00C0017
:1087A0001810000420000200000000000020000259
:1087B0001000040C00180780F001FFC0007F0000CB
:1087C00000000000000000000000000000000000A9
:1087D00000004200006600006600003C0000180037
:1087E00003FFC0001800003C0000660000660000A7
:1087F0004200000000000800000800000800000817
:108800000000080001FFC000080000080000080088
:108810000008000008000000000000010000310016
:10882000003200001C0000000000000000000000FA
:108830000000000000000000000000000000080030
:108840000008000008000008000008000008000000
:1088500008000008000008000008000000000000F8
:108860000000000000003800003800003800000060
:1088700000000000000000000000000000000000F8
:10888000000000000000000600001C000070000155
:1088900080000E0000380000C0000700001C00002F
:1088A000300000000000000000007F8001FFE003B6
:1088B00080700600180400080400080600180380F1
:1088C0007001FFE0007F8000000000000000000059
:1088D00001000801000801000803FFF807FFF80085
:1088E0000008000008000008000000000000000070
:1088F0000001C03802C0580400980401180402188E
:10890000040418061C1803F81801E0F80000000021
:10891000000000000001C0E003C0F00400080408EB
:108920000804080806180803F41801E7F00001E03D
:10893000000000000000000000000300000D000027
:10894000110000610000810803010807FFF80FFF14
:10895000F80001080001080000000000000000E02D
:1089600007FCD006080806100806100806100806BE
:108970001838060FF00607C00000000000000000D5
:1089800000003F8001FFE003843002081804100853
:10899000041008041008071810030FF00007C000A7
:1089A000000000000000000003C0000700000600F7
:1089B000000600F80607F806180006E000070000A9
:1089C00006000000000000000001E1E003F7F006EF
:1089D0003410041808041808040C08040C080616BF
:1089E0001803F3F001C1E000000000000000F800EF
:1089F00003FC3003063804020804020804020804D9
:108A000004100308F001FFC0007F00000000000018
:108A100000000000000000000000000000007038AE
:108A200000703800703800000000000000000000F6
:108A30000000000000000000000000000000000036
:108A40000000301A00301C00000000000000000090
:108A5000000000000000000000000000000800000E
:108A6000140000220000410000808001004002004C
:108A70002004001008000800000000000000210091
:108A80000021000021000021000021000021000041
:108A90002100002100002100002100000000000052
:108AA000000000000800080400100200200100403F
:108AB0000080800041000022000014000008000037
:108AC000000000000003C00004C000040000080013
:108AD00038080F380808380810000C300007E0008C
:108AE00003C000000000000000003F8000FFE00322
:108AF0008070020F1006708804C088048308047F09
:108B00008802C09003012000FE4000000800001809
:108B10000001F8003E0801C20007020007E2000061
:108B2000FE00001FC80001F8000038000008040023
:108B30000807FFF807FFF8040808040808040808F5
:108B400004080806180803F41801E7F00001E00023
:108B50000000000000003F8001FFE0038070020081
:108B6000180400080400080400080400100600208F
:108B70000780C000000004000807FFF807FFF804A2
:108B80000008040008040008040018020010038014
:108B90007001FFE0007F8000000004000807FFF87C
:108BA00007FFF80408080408080408080408080473
:108BB0003E080400080600180100600000000400E0
:108BC0000807FFF807FFF804080804080004080075
:108BD000040800043E0006000006000001800000BA
:108BE0000000000000003F8001FFE00380700600ED
:108BF000180400080402080402080203F00783F0C6
:108C000000020000020004000807FFF807FFF80454
:108C10000808000800000800000800000800040818
:108C20000807FFF807FFF804000800000000000034
:108C300004000804000804000807FFF807FFF80410
:108C40000008040008040008000000000000000004
:108C500000000006000007000001040001040001FC
:108C600004000307FFFE07FFFC04000004000004EB
:108C7000000004000807FFF807FFF8040C080018BC
:108C800000003E0004C7800503C80600F804003851
:108C900004001800000804000807FFF807FFF804A4
:108CA000000800000800000800000800000800009C
:108CB0000800001800006000000004000807FFF82A
:108CC00007800807FC00007FC00003F80007C00011
:108CD000780007800807FFF807FFF8040008040081
:108CE0000807FFF807000803C00000E00000380094
:108CF000001E000007000001C00400F007FFF80498
:108D00000000000000007F8001FFE003807006008B
:108D10001804000804000806001803003001FFE0F2
:108D2000007F8000000004000807FFF807FFF80438
:108D30000408040400040400040400040400060CF5
:108D40000003F80001F000000000000000007F8038
:108D500001FFE00380700600880400880400C80654
:108D6000003C03003E01FFE6007F84000000040099
:108D70000807FFF807FFF8040808040800040C00BF
:108D8000040F00040BC00610F003F03801E00800E7
:108D9000000800000001E0F803F03006301004186D
:108DA00008041808040C08040C080206180207F04E
:108DB0000781E000000001800006000004000004BC
:108DC000000004000807FFF807FFF804000804008B
:108DD0000004000006000001800004000007FFE01E
:108DE00007FFF00400180000080000080000080059
:108DF000000800000804001007FFE0040000040061
:108E00000006000007E00007FE00041FE00001F874
:108E10000000380001E0043E0007C0000600000426
:108E2000000004000007E00007FFC0041FF800076F
:108E3000C007F80007FF80043FF80007C004F800EF
:108E400007000004000000000004000806001807E6
:108E5000C07805F1C8003E00001F800463E8078069
:108E6000F8060018040008000000040000060000D6
:108E700007800007E008047C08001FF80007F800DE
:108E8000180804E0080700000600000400000000C5
:108E9000000100080600380400F80403E8040F0885
:108EA000047C0805F00807C00807001804006000EB
:108EB00000000000000000000000000000000000B2
:108EC000003FFFFE200002200002200002200002DE
:108ED0002000020000000000000000000800000761
:108EE000000000C0000038000006000001C00000C3
:108EF0003000000E00000100000000000000000033
:108F00002000022000022000022000022000023F78
:108F1000FFFE000000000000000000000000000054
:108F200000000000000000080000100000300000F9
:108F300020000030000010000008000000000000C9
:108F4000000000000100000100000100000100001D
:108F5000010000010000010000010000010000010B
:108F600000000100000100000000000000000020DF
:108F700000002000001000001000000000000000B1
:108F8000000000000000000000000000000000F0F1
:108F90000019F8001B180022080026080024080009
:108FA0002410003FF8001FF800000800001800001F
:108FB0000004000007FFF80FFFF000181800100869
:108FC000002008002008003018001FF0000FC0002B
:108FD00000000000000007C0001FF0001830002053
:108FE00008002008002008003C08001C1000006059
:108FF0000000000000000000000007C0001FF0009B
:10900000381800200800200800200804101007FF6E
:10901000F80FFFF00000100000000000000000004A
:109020000007C0001FF000123000221800220800C4
:109030002208003208001E10000E20000000000070
:109040000000200000200800200801FFF803FFF8BE
:109050000620080420080420080720000300000060
:10906000000000000000000E000E6E001FF3003133
:10907000B10020B10020B1003191001F13002E1E5D
:1090800000200E00300000000004000807FFF80F69
:10909000FFF8001008002000002000002008003F1A
:1090A000F8001FF8000008000000000000000000A9
:1090B000002008002008002008063FF8063FF800BE
:1090C0000008000008000008000000000000000088
:1090D0000000000000000300000300200100200148
:1090E000002003063FFE063FFC00000000000000D9
:1090F000000000000004000807FFF80FFFF800015F
:1091000088000300002FC00038F800203800200835
:109110000000080000000000000000000400080437
:10912000000804000807FFF80FFFF800000800001F
:1091300008000008000000000000002008003FF8C0
:10914000003FF8001008002000003FF8003FF80042
:109150001008002000003FF8003FF8000008000061
:1091600000002008003FF8003FF800100800100041
:10917000002000002008003FF8001FF80000080051
:1091800000000000000007C0000FF00018300030A1
:1091900008002008002008003008001830000FF0F8
:1091A0000007C0000000000000002001003FFF0099
:1091B0003FFF0010110020090020080020080030A7
:1091C00038001FF0000FC00000000000000007C0C2
:1091D000001FF000381800200800200800200900B7
:1091E0001011001FFF003FFF0000010000000020E1
:1091F00008002008002008003FF8003FF800080899
:10920000001008002008002000003000003000009E
:109210000000000000000000000C78001E18003361
:10922000080023080021080021880021980030F060
:109230000038600000000000000020000020000056
:10924000200000FFF003FFF80020080020080020A5
:1092500008000030000000000000000000002000B6
:10926000003FF0007FF80000180000080000080030
:109270002010003FF8007FF0000010000000000008
:1092800000002000003000003C00003F800023F080
:10929000000078000070002380003C0000300000D7
:1092A0002000002000003C00003FE00023F8000008
:1092B000E0002700003E00003FE00021F80001E050
:1092C000003E0000200000000000200800200800F0
:1092D0003838003E680027800003C8002CF80038AA
:1092E00038002018002008000000000000002000C6
:1092F000003003003C01003F830023EC00007000BD
:109300002380003C0000200000200000000000003E
:10931000000000000038080020380020F80023E892
:10932000002F88003E080038080020180000700058
:10933000000000000000000000000000000000002D
:10934000000008000014001FF7FC30000620000297
:10935000000000000000000000000000000000000D
:109360000000000000000000FFFFFF000000000000
:1093700000000000000000000000000000000000ED
:109380002000023000061FF7FC0014000008000057
:1093900000000000000000000000000000000000CD
:1093A00000180000600000400000400000200000A5
:1093B0001000000800000400000400000C00001071
:1093C000000000000000000000000000000000009D
:1093D000000000000000000000000000000000008D
:1093E000000000000000000000000000000000007D
:1093F000000000000000000000000000000000006D
:10940000000000000000000000000000000000005C
:10941000000000000000000000000000000000004C
:10942000000000000000000000000000000000003C
:10943000000000000000000000000000000000002C
:10944000000000000000000000000000000000001C
:109450000000000000000000000007F000C007FF4F
:10946000E1E007F001E0000000C0000000000000A3
:1094700000000000000000000000000000000000EC
:1094800000000000000000000000000000000000DC
:1094900000000000000000000000000000000000CC
:1094A00000000000000000000000000000000000BC
:1094B00000000000000000000000000000000000AC
:1094C000000000000000000000000020000001C0BB
:1094D0000000078000001F0000001E0000001C208C
:1094E000000001C00000078000001F0000001E00F7
:1094F00000001C0000000000000000000000000050
:10950000000000000000000000000000000000005B
:10951000000000000000000000000000000000004B
:10952000000000000000000000000000000000003B
:10953000000000000000000000000000000000002B
:1095400000000000000000180C0000180C000018BB
:109550000FE0001FFC0003F80C0000180C000018BE
:109560000C0000180C0000180C0000180FE0001F81
:10957000FC0003F80C0000180C0000180C000000A0
:1095800000000000000000000000000000000000DB
:1095900000000000000000000000000000000000CB
:1095A00000000000000000000000000000000000BB
:1095B00000000000000000000000000000000000AB
:1095C000000000000000000000000000078000789C
:1095D00007C000FC0640010E002003070020020324
:1095E00080200FFFFFFC0201C0200200E06001307C
:1095F000704001F03F8000F01F00000000000000FC
:10960000000000000000000000000000000000005A
:10961000000000000000000000000000000000004A
:10962000000000000000000000000000000000003A
:10963000000000000000000000000000000000002A
:10964000000000FE000001FF000003018000020096
:109650008060030181C001FF070000FE18000000C8
:10966000E0000003BF00000CFFC00071806001C17A
:109670000020030180600000FFC000003F000000E8
:1096800000000000000000000000000000000000DA
:1096900000000000000000000000000000000000CA
:1096A00000000000000000000000000000000000BA
:1096B00000000000000000000000000000000000AA
:1096C000000000001F0000007FC000FCC0C001FFC0
:1096D00080600303E0200202782002061E2003FCC3
:1096E000074001F00380000103C000011C6000017D
:1096F000E020000100200001004000000180000087
:109700000000000000000000000000000000000059
:109710000000000000000000000000000000000049
:109720000000000000000000000000000000000039
:109730000000000000000000000000000000000029
:10974000000000000000002000001C6000001C4021
:1097500000001F8000000F0000000000000000005B
:1097600000000000000000000000000000000000F9
:1097700000000000000000000000000000000000E9
:1097800000000000000000000000000000000000D9
:1097900000000000000000000000000000000000C9
:1097A00000000000000000000000000000000000B9
:1097B00000000000000000000000000000000000A9
:1097C0000000000000000000000000000000000099
:1097D0000000000000000000000000000000000782
:1097E000F800003FFF00007807C001C000E0030060
:1097F000003004000008080000041000000200000F
:109800000000000000000000000000000000000058
:109810000000000000000000000000000000000048
:109820000000000000000000000000000000000038
:109830000000000000000000000000000000000028
:1098400000000000000010000002080000040400F6
:1098500000080300003001C000E0007807C0003FAE
:10986000FF000007F80000000000000000000000FA
:1098700000000000000000000000000000000000E8
:1098800000000000000000000000000000000000D8
:1098900000000000000000000000000000000000C8
:1098A00000000000000000000000000000000000B8
:1098B00000000000000000000000000000000000A8
:1098C00000000000000000000000000C1800000E66
:1098D0003800000E38000006300000036000006110
:1098E000438000FFFF80006143000003600000062A
:1098F0003000000E3800000E3800000C1800000088
:109900000000000000000000000000000000000057
:109910000000000000000000000000000000000047
:109920000000000000000000000000000000000037
:109930000000000000000000000000000000000027
:109940000000000000000000000000008000000097
:109950008000000080000000800000008000000007
:109960008000007FFF0000008000000080000000F9
:1099700080000000800000008000000080000000E7
:1099800000000000000000000000000000000000D7
:1099900000000000000000000000000000000000C7
:1099A00000000000000000000000000000000000B7
:1099B00000000000000000000000000000000000A7
:1099C00000000000000000000001000000E30000B3
:1099D00000E2000000FC0000007800000000000031
:1099E0000000000000000000000000000000000077
:1099F0000000000000000000000000000000000067
:109A00000000000000000000000000000000000056
:109A10000000000000000000000000000000000046
:109A20000000000000000000000000000000000036
:109A30000000000000000000000000000000000026
:109A40000000000000000000800000008000000016
:109A50008000000080000000800000008000000006
:109A600080000000800000008000000080000000F6
:109A700080000000800000008000000080000000E6
:109A800000000000000000000000000000000000D6
:109A900000000000000000000000000000000000C6
:109AA00000000000000000000000000000000000B6
:109AB00000000000000000000000000000000000A6
:109AC00000000000000000000000000000C00000D6
:109AD00001E0000001E0000000C000000000000004
:109AE0000000000000000000000000000000000076
:109AF0000000000000000000000000000000000066
:109B00000000000000000000000000000000000055
:109B10000000000000000000000000000000000045
:109B20000000000000000000000000000000000035
:109B30000000000000000000000000000000000025
:109B40000000000000000000000C000000380000D1
:109B500000E00000038000000E000000380000005C
:109B6000E00000038000000E00000038000000E06C
:109B70000000038000000E0000001800000000003C
:109B800000000000000000000000000000000000D5
:109B900000000000000000000000000000000000C5
:109BA00000000000000000000000000000000000B5
:109BB00000000000000000000000000000000000A5
:109BC00000000000000000000000000FF800007F0F
:109BD000FF0000F00780018000C003000060020069
:109BE000002002000020020000200300006001802D
:109BF00000C000E00380007FFF00000FF8000000BD
:109C00000000000000000000000000000000000054
:109C10000000000000000000000000000000000044
:109C20000000000000000000000000000000000034
:109C30000000000000000000000000000000000024
:109C40000000000000000000000000000000008094
:109C5000002000800020008000200080006001FFC4
:109C6000FFE003FFFFE000000060000000200000B4
:109C700000200000002000000000000000000000A4
:109C800000000000000000000000000000000000D4
:109C900000000000000000000000000000000000C4
:109CA00000000000000000000000000000000000B4
:109CB00000000000000000000000000000000000A4
:109CC00000000000000000000000007800E00098A4
:109CD00001600100026002000460020008600200EE
:109CE0001060020020600200406003008060018379
:109CF000006001FE00E0007C078000000000000022
:109D00000000000000000000000000000000000053
:109D10000000000000000000000000000000000043
:109D20000000000000000000000000000000000033
:109D30000000000000000000000000000000000023
:109D40000000000000000000000000F0078001F0AB
:109D500007C00100004002000020020100200201B3
:109D6000002002010020030380200186804001FCC6
:109D7000C0C000787F8000001E00000000000000CE
:109D800000000000000000000000000000000000D3
:109D900000000000000000000000000000000000C3
:109DA00000000000000000000000000000000000B3
:109DB00000000000000000000000000000000000A3
:109DC0000000000000000000080000003800000053
:109DD00048000001880000060800000C0810003050
:109DE00008100040081001FFFFF003FFFFF003FF21
:109DF000FFF000000810000008100000081000002C
:109E00000000000000000000000000000000000052
:109E10000000000000000000000000000000000042
:109E20000000000000000000000000000000000032
:109E30000000000000000000000000000000000022
:109E40000000000000000000000000000780001F6C
:109E5000864003E1002003020020030400200304E5
:109E60000020030400200304002003060040030335
:109E700001C00301FF8003007E000000000000001D
:109E800000000000000000000000000000000000D2
:109E900000000000000000000000000000000000C2
:109EA00000000000000000000000000000000000B2
:109EB00000000000000000000000000000000000A2
:109EC000000000000000000000000007FC00003F50
:109ED000FF000070C380008180C0010100600302A8
:109EE00000200202002002020020020200200203E1
:109EF000004001C180C000C0FF8000007E00000063
:109F00000000000000000000000000000000000051
:109F10000000000000000000000000000000000041
:109F20000000000000000000000000000000000031
:109F30000000000000000000000000000000000021
:109F40000000000000000000000000F0000003C05E
:109F500000000380000003000000030007E003008E
:109F60003FE00301C0000306000003180000036087
:109F7000000003800000030000000000000000005B
:109F800000000000000000000000000000000000D1
:109F900000000000000000000000000000000000C1
:109FA00000000000000000000000000000000000B1
:109FB00000000000000000000000000000000000A1
:109FC00000000000000000001F0000783F8000FC3F
:109FD00060C0018EC0400307802002030020020100
:109FE0008020020180200201C0200301E0400186A0
:109FF00070C000FC3F8000781F00000000000000DF
:10A000000000000000000000000000000000000050
:10A010000000000000000000000000000000000040
:10A020000000000000000000000000000000000030
:10A030000000000000000000000000000000000020
:10A04000000000000000003F000000FF81C001C0D0
:10A05000C1C0010060200200202002002020020078
:10A06000202002002060020040C00100C18000C129
:10A070008F00007FFE00001FF000000000000000C5
:10A0800000000000000000000000000000000000D0
:10A0900000000000000000000000000000000000C0
:10A0A00000000000000000000000000000000000B0
:10A0B00000000000000000000000000000000000A0
:10A0C0000000000000000000000000000000000090
:10A0D00000000000000000000000000300C00007B6
:10A0E00081E0000781E0000300C0000000000000E4
:10A0F0000000000000000000000000000000000060
:10A10000000000000000000000000000000000004F
:10A11000000000000000000000000000000000003F
:10A12000000000000000000000000000000000002F
:10A13000000000000000000000000000000000001F
:10A14000000000000000000000000000000000000F
:10A15000000000000000000000000006006600068D
:10A160000078000000000000000000000000000077
:10A1700000000000000000000000000000000000DF
:10A1800000000000000000000000000000000000CF
:10A1900000000000000000000000000000000000BF
:10A1A00000000000000000000000000000000000AF
:10A1B000000000000000000000000000000000009F
:10A1C000000000000000000000000000800000010E
:10A1D000C0000003600000063000000C18000018EA
:10A1E0000C00003006000060030000C00180010088
:10A1F00000400200002004000010000000000000E9
:10A20000000000000000000000000000000000004E
:10A21000000000000000000000000000000000003E
:10A22000000000000000000000000000000000002E
:10A23000000000000000000000000000000000001E
:10A2400000000000000000041000000410000004E2
:10A2500010000004100000041000000410000004AE
:10A26000100000041000000410000004100000049E
:10A270001000000410000004100000041000000092
:10A2800000000000000000000000000000000000CE
:10A2900000000000000000000000000000000000BE
:10A2A00000000000000000000000000000000000AE
:10A2B000000000000000000000000000000000009E
:10A2C0000000000000000000000004000010020078
:10A2D00000200100004000C0018000600300003049
:10A2E000060000180C00000C1800000630000003E7
:10A2F00060000001C00000008000000000000000BD
:10A30000000000000000000000000000000000004D
:10A31000000000000000000000000000000000003D
:10A32000000000000000000000000000000000002D
:10A33000000000000000000000000000000000001D
:10A34000000000000000000000000078000001F89C
:10A3500000000238000002000000040000C00400F9
:10A3600079E0040081E0040100C00403000002025F
:10A3700000000306000001FC000000F800000000DF
:10A3800000000000000000000000000000000000CD
:10A3900000000000000000000000000000000000BD
:10A3A00000000000000000000000000000000000AD
:10A3B000000000000000000000000000000000009D
:10A3C000000000000000000FF800003FFE000070D9
:10A3D000078000C000C00101F8400307FC20021EF6
:10A3E00004200230082002203020023FFC20013FE0
:10A3F000044001800CC000E03180001FC20000005A
:10A40000000000000000000000000000000000004C
:10A41000000000000000000000000000000000003C
:10A42000000000000000000000000000000000002C
:10A43000000000000000000000000000000000001C
:10A4400000000000002000000060000003E00000A9
:10A450003E200003E020003E200003E020000380B7
:10A46000200007FC2000003FE0000003FE20000069
:10A470003FE0000001E0000000200000002000009C
:10A4800000000000000000000000000000000000CC
:10A4900000000000000000000000000000000000BC
:10A4A00000000000000000000000000000000000AC
:10A4B000000000000000000000000000000000009C
:10A4C000000000000000020000200200002003FF46
:10A4D000FFE003FFFFE00201002002010020020173
:10A4E0000020020100200201002003030020018659
:10A4F000806001FCC0C000F87F8000001F000000E9
:10A50000000000000000000000000000000000004B
:10A51000000000000000000000000000000000003B
:10A52000000000000000000000000000000000002B
:10A53000000000000000000000000000000000001B
:10A540000000000000000007F800003FFF0000705E
:10A55000078000C000C0010000400300002002008E
:10A560000020020000200200002002000020010064
:10A570000040018000C003C00180003006000000E0
:10A5800000000000000000000000000000000000CB
:10A5900000000000000000000000000000000000BB
:10A5A00000000000000000000000000000000000AB
:10A5B000000000000000000000000000000000009B
:10A5C000000000000000020000200200002003FF45
:10A5D000FFE003FFFFE00200002002000020020075
:10A5E0000020020000200300006001000040018004
:10A5F00000C000F00780007FFE00000FF8000000A0
:10A60000000000000000000000000000000000004A
:10A61000000000000000000000000000000000003A
:10A62000000000000000000000000000000000002A
:10A63000000000000000000000000000000000001A
:10A64000000000000000020000200200002003FFC4
:10A65000FFE003FFFFE002010020020100200201F1
:10A660000020020100200201002002038020020FCE
:10A67000E0200300006003C000E000600300000071
:10A6800000000000000000000000000000000000CA
:10A6900000000000000000000000000000000000BA
:10A6A00000000000000000000000000000000000AA
:10A6B000000000000000000000000000000000009A
:10A6C000000000000000020000200200002003FF44
:10A6D000FFE003FFFFE00201002002010020020171
:10A6E000000002010000020100000201000002035C
:10A6F0008000030FE0000300000003C000000060C2
:10A700000000000000000000000000000000000049
:10A710000000000000000000000000000000000039
:10A720000000000000000000000000000000000029
:10A730000000000000000000000000000000000019
:10A740000000000000000007F800003FFE0000705D
:10A75000078001C001C0010000400300002002008A
:10A760000020020000200200002001002020010043
:10A77000204003C03F8000303F80000020000000E8
:10A7800020000000000000000000000000000000A9
:10A7900000000000000000000000000000000000B9
:10A7A00000000000000000000000000000000000A9
:10A7B0000000000000000000000000000000000099
:10A7C0000000020000200200002003FFFFE003FF62
:10A7D000FFE00200802002008020000080000000D6
:10A7E000800000008000020080200200802003FF23
:10A7F000FFE003FFFFE00200002002000020000055
:10A800000000000000000000000000000000000048
:10A810000000000000000000000000000000000038
:10A820000000000000000000000000000000000028
:10A830000000000000000000000000000000000018
:10A840000000000000000000000000000000020006
:10A85000002002000020020000200200002003FF70
:10A86000FFE003FFFFE002000020020000200200E2
:10A870000020020000200000000000000000000096
:10A8800000000000000000000000000000000000C8
:10A8900000000000000000000000000000000000B8
:10A8A00000000000000000000000000000000000A8
:10A8B0000000000000000000000000000000000098
:10A8C0000000000000000000000E0000000F00006B
:10A8D000000F000000010200000102000001020060
:10A8E00000030200000603FFFFFC03FFFFF8020065
:10A8F0000000020000000200000002000000000052
:10A900000000000000000000000000000000000047
:10A910000000000000000000000000000000000037
:10A920000000000000000000000000000000000027
:10A930000000000000000000000000000000000017
:10A94000000000000000020000200200002003FFC1
:10A95000FFE003FFFFE00200C0200201002000072B
:10A960008000000FE0000030F80002603E2003800D
:10A970000F20030003E0020000E0020000200000BE
:10A9800000200000000000000000000000000000A7
:10A9900000000000000000000000000000000000B7
:10A9A00000000000000000000000000000000000A7
:10A9B0000000000000000000000000000000000097
:10A9C000000000000000020000200200002003FF41
:10A9D000FFE003FFFFE00200002002000020000073
:10A9E00000200000002000000020000000200000E7
:10A9F000002000000060000000E0000003000000F4
:10AA00000000000000000000000000000000000046
:10AA10000000000000000000000000000000000036
:10AA20000000000000000000000000000000000026
:10AA30000000000000000000000000000000000016
:10AA40000000020000200200002003FFFFE003E0FE
:10AA5000002003FF0020001FF0000001FF80000025
:10AA60000FE000001E000003E000003E002003E0B5
:10AA7000002003FFFFE003FFFFE0020000200200D0
:10AA800000200000000000000000000000000000A6
:10AA900000000000000000000000000000000000B6
:10AAA00000000000000000000000000000000000A6
:10AAB0000000000000000000000000000000000096
:10AAC0000000020000200200002003FFFFE00380DE
:10AAD000002003F0002000FC0000001F0000000721
:10AAE000C0000001F00000007C0002001F80020096
:10AAF00007E003FFFFE0020000000200000000008A
:10AB00000000000000000000000000000000000045
:10AB10000000000000000000000000000000000035
:10AB20000000000000000000000000000000000025
:10AB30000000000000000000000000000000000015
:10AB4000000000000000000FF800003FFE0000F0D1
:10AB50000780018000C001000040020000200200C8
:10AB600000200200002002000020010000400180BF
:10AB700000C000F00380003FFE00000FF80000005E
:10AB800000000000000000000000000000000000C5
:10AB900000000000000000000000000000000000B5
:10ABA00000000000000000000000000000000000A5
:10ABB0000000000000000000000000000000000095
:10ABC000000000000000020000200200002003FF3F
:10ABD000FFE003FFFFE0020080200200802002006F
:10ABE000800002008000020080000200800003015B
:10ABF00080000183000000FE0000007C00000000D7
:10AC00000000000000000000000000000000000044
:10AC10000000000000000000000000000000000034
:10AC20000000000000000000000000000000000024
:10AC30000000000000000000000000000000000014
:10AC4000000000000000000FF800007FFF0000F08F
:10AC50000380018001C001000640020004200200C0
:10AC6000042002000620020003E0010000F8018039
:10AC7000005C00E0038C003FFF0C000FFC1800009C
:10AC800000000000000000000000000000000000C4
:10AC900000000000000000000000000000000000B4
:10ACA00000000000000000000000000000000000A4
:10ACB0000000000000000000000000000000000094
:10ACC000000000000000020000200200002003FF3E
:10ACD000FFE003FFFFE0020100200201002002016B
:10ACE00080000201E0000201FC0003033F800186B6
:10ACF00007E001FC00E000F8002000000020000058
:10AD00000000000000000000000000000000000043
:10AD10000000000000000000000000000000000033
:10AD20000000000000000000000000000000000023
:10AD30000000000000000000000000000000000013
:10AD4000000000000000000000000078060000FE87
:10AD500001E0018600C0030300400203002002015D
:10AD60008020020180200201C0200200C0200100DA
:10AD7000E060018070C003E03F8000001F00000021
:10AD800000000000000000000000000000000000C3
:10AD900000000000000000000000000000000000B3
:10ADA00000000000000000000000000000000000A3
:10ADB0000000000000000000000000000000000093
:10ADC000000000000000006000000380000003009D
:10ADD000000002000000020000200200002003FF2B
:10ADE000FFE003FFFFE0020000200200002002005D
:10ADF0000000020000000380000000E000000000EE
:10AE00000000000000000000000000000000000042
:10AE10000000000000000000000000000000000032
:10AE20000000000000000000000000000000000022
:10AE30000000000000000000000000000000000012
:10AE40000000020000000200000003FFFF0003FFFB
:10AE5000FFC002000040020000600000002000006F
:10AE6000002000000020000000200200004002003E
:10AE7000008003FFFF00020000000200000000004D
:10AE800000000000000000000000000000000000C2
:10AE900000000000000000000000000000000000B2
:10AEA00000000000000000000000000000000000A2
:10AEB0000000000000000000000000000000000092
:10AEC000000000000000020000000200000003C0BB
:10AED000000003FC0000023FC0000003F800000077
:10AEE0007F80000007E00000078000007800020378
:10AEF000C000023C000003C000000200000002008D
:10AF00000000000000000000000000000000000041
:10AF10000000000000000000000000000000000031
:10AF20000000000000000000000000000000000021
:10AF30000000000000000000000000000000000011
:10AF400000000200000003C0000003FF8000023F79
:10AF5000FE0002007FE000000F000200F00003EF9F
:10AF6000000003FF8000020FFE0000003FE0000031
:10AF70001F000207E00003F80000030000000200C9
:10AF800000000000000000000000000000000000C1
:10AF900000000000000000000000000000000000B1
:10AFA00000000000000000000000000000000000A1
:10AFB0000000000000000000000000000000000091
:10AFC00000000000000002000020020000200380BA
:10AFD00000E003F0032002FC0C20021F30000007F9
:10AFE000C0000007F00002187C0002601F200380F0
:10AFF00003E0020000E0020000200000002000004A
:10B000000000000000000000000000000000000040
:10B010000000000000000000000000000000000030
:10B020000000000000000000000000000000000020
:10B030000000000000000000000000000000000010
:10B04000000000000000020000000300000003C038
:10B05000000003F80000023E0020020FC0200001A3
:10B06000FFE000007FE000038020021C002002704F
:10B070000000038000000200000002000000000049
:10B0800000000000000000000000000000000000C0
:10B0900000000000000000000000000000000000B0
:10B0A00000000000000000000000000000000000A0
:10B0B0000000000000000000000000000000000090
:10B0C00000000000000000000020006000E003809D
:10B0D00003E003000FA002003E200200F82002035C
:10B0E000E020020F8020023E00200278002003E0D2
:10B0F0000060038000E00200030000000000000088
:10B10000000000000000000000000000000000003F
:10B11000000000000000000000000000000000002F
:10B12000000000000000000000000000000000001F
:10B13000000000000000000000000000000000000F
:10B1400000000000000000000000000000000000FF
:10B15000000000000000000000001FFFFFFC1000C6
:10B16000000410000004100000041000000410008F
:10B1700000041000000410000004000000000000A3
:10B1800000000000000000000000000000000000BF
:10B1900000000000000000000000000000000000AF
:10B1A000000000000000000000000000000000009F
:10B1B000000000000000000000000000000000008F
:10B1C0000000000000000000000000000000070078
:10B1D000000003C0000000780000001E0000000313
:10B1E000C0000000F00000001E000000078000000A
:10B1F00000F00000003C000000060000000000001D
:10B20000000000000000000000000000000000003E
:10B21000000000000000000000000000000000002E
:10B22000000000000000000000000000000000001E
:10B23000000000000000000000000000000000000E
:10B2400000000000000000000000100000041000DA
:10B25000000410000004100000041000000410009E
:10B260000004100000041FFFFFFC000000000000AD
:10B2700000000000000000000000000000000000CE
:10B2800000000000000000000000000000000000BE
:10B2900000000000000000000000000000000000AE
:10B2A000000000000000000000000000000000009E
:10B2B000000000000000000000000000000000008E
:10B2C000000000000000000000000000000000007E
:10B2D0000000020000000400000008000000180048
:10B2E000000010000000180000001800000004001A
:10B2F000000002000000000000000000000000004C
:10B30000000000000000000000000000000000003D
:10B31000000000000000000000000000000000002D
:10B32000000000000000000000000000000000001D
:10B33000000000000000000000000000000000000D
:10B3400000000000000100000001000000010000FA
:10B3500000010000000100000001000000010000E9
:10B3600000010000000100000001000000010000D9
:10B3700000010000000100000001000000010000C9
:10B3800000010000000000000000000000000000BC
:10B3900000000000000000000000000000000000AD
:10B3A000000000000000000000000000000000009D
:10B3B000000000000000000000000000000000008D
:10B3C000000000000000000000000000000010006D
:10B3D000000010000000100000001800000008002D
:10B3E0000000040000000000000000000000000059
:10B3F000000000000000000000000000000000004D
:10B40000000000000000000000000000000000003C
:10B41000000000000000000000000000000000002C
:10B42000000000000000000000000000000000001C
:10B43000000000000000000000000000000000000C
:10B440000000000000000000038000018FC0000326
:10B450008C60000618200004102000041020000456
:10B46000202000042040000620400003FFC000010F
:10B47000FFE00000002000000020000000C00000ED
:10B4800000000000000000000000000000000000BC
:10B4900000000000000000000000000000000000AC
:10B4A000000000000000000000000000000000009C
:10B4B000000000000000000000000000000000008C
:10B4C000000000000000020000000200000003FF76
:10B4D000FFE007FFFFC0000180C000020060000223
:10B4E00000200004002000040020000400200006CA
:10B4F0000040000300C00001FF800000FE000000CB
:10B50000000000000000000000000000000000003B
:10B51000000000000000000000000000000000002B
:10B52000000000000000000000000000000000001B
:10B53000000000000000000000000000000000000B
:10B540000000000000000000000000007E0000017C
:10B55000FF80000381C000020040000600200004BC
:10B56000002000040020000400200006002000034A
:10B57000C0400001C0800000030000000000000087
:10B5800000000000000000000000000000000000BB
:10B5900000000000000000000000000000000000AB
:10B5A000000000000000000000000000000000009B
:10B5B000000000000000000000000000000000008B
:10B5C0000000000000000000000000007E000001FC
:10B5D000FF80000380C0000600600004002000041B
:10B5E000002000040020020400400202008003FF4B
:10B5F000FFE007FFFFC00000004000000040000027
:10B60000000000000000000000000000000000003A
:10B61000000000000000000000000000000000002A
:10B62000000000000000000000000000000000001A
:10B63000000000000000000000000000000000000A
:10B640000000000000000000000000007E0000017B
:10B65000FF80000311C000021040000410600004CD
:10B660001020000410200004102000061020000309
:10B6700010400001F0C00000710000000000000058
:10B6800000000000000000000000000000000000BA
:10B6900000000000000000000000000000000000AA
:10B6A000000000000000000000000000000000009A
:10B6B000000000000000000000000000000000008A
:10B6C0000000000000000000000000040000000472
:10B6D00000200004002000040020007FFFE001FFA4
:10B6E000FFE0010400200304002002040020020403
:10B6F0000020020400000200000001C0000001C0A0
:10B700000000000000000000000000000000000039
:10B710000000000000000000000000000000000029
:10B720000000000000000000000000000000000019
:10B730000000000000000000000000000000000009
:10B74000000000000000000000000000001C0000DD
:10B75000E33E0003FFC200020CC3000404C1000466
:10B7600004C1000404C1000404C100060CC10003AC
:10B77000F8C30005F0620006007E0006003C0000F1
:10B7800000000000000000000000000000000000B9
:10B7900000000000000000000000000000000000A9
:10B7A0000000000000000000000000000000000099
:10B7B0000000000000000000000000000000000089
:10B7C000000000000000020000200200002003FF33
:10B7D000FFE007FFFFE0000100200002002000065C
:10B7E0000000000400000004000000040020000627
:10B7F00000200003FFE00001FFE000000020000047
:10B800000020000000000000000000000000000018
:10B810000000000000000000000000000000000028
:10B820000000000000000000000000000000000018
:10B830000000000000000000000000000000000008
:10B8400000000000000000000000000000000004F4
:10B8500000200004002000040020000400200387D2
:10B86000FFE0038FFFE003800020000000200000C5
:10B870000020000000200000000000000000000088
:10B8800000000000000000000000000000000000B8
:10B8900000000000000000000000000000000000A8
:10B8A0000000000000000000000000000000000098
:10B8B0000000000000000000000000000000000088
:10B8C0000000000000000000000000000000000078
:10B8D0000006000000070000000100000001000455
:10B8E00000010004000100040003000400060387B7
:10B8F000FFFC038FFFF80380000000000000000041
:10B900000000000000000000000000000000000037
:10B910000000000000000000000000000000000027
:10B920000000000000000000000000000000000017
:10B930000000000000000000000000000000000007
:10B94000000000000000020000200200002003FFB1
:10B95000FFE007FFFFE000000820000010200000CB
:10B9600030000000FC0000058E00000707A0000664
:10B9700001E0000400E000040020000000200000BE
:10B9800000000000000000000000000000000000B7
:10B9900000000000000000000000000000000000A7
:10B9A0000000000000000000000000000000000097
:10B9B0000000000000000000000000000000000087
:10B9C0000000000000000000000000000000020075
:10B9D000002002000020020000200200002003FFDF
:10B9E000FFE007FFFFE00000002000000020000053
:10B9F0000020000000200000000000000000000007
:10BA00000000000000000000000000000000000036
:10BA10000000000000000000000000000000000026
:10BA20000000000000000000000000000000000016
:10BA30000000000000000000000000000000000006
:10BA4000000000000000000400200007FFE0000FDD
:10BA5000FFE00002002000040000000400200007B6
:10BA6000FFE00003FFE000020020000400000004EB
:10BA700000200007FFE00003FFE0000000200000BE
:10BA800000000000000000000000000000000000B6
:10BA900000000000000000000000000000000000A6
:10BAA0000000000000000000000000000000000096
:10BAB0000000000000000000000000000000000086
:10BAC0000000000000000004002000040020000727
:10BAD000FFE0000FFFE00001002000020020000254
:10BAE0000000000400000004000000040020000624
:10BAF00000200003FFE00001FFE000000020000044
:10BB00000020000000000000000000000000000015
:10BB10000000000000000000000000000000000025
:10BB20000000000000000000000000000000000015
:10BB30000000000000000000000000000000000005
:10BB40000000000000000000000000007E00000077
:10BB5000FF80000381C000020040000600200004B6
:10BB60000020000400200004002000060020000245
:10BB70000040000381C00001FF8000007E00000043
:10BB800000000000000000000000000000000000B5
:10BB900000000000000000000000000000000000A5
:10BBA0000000000000000000000000000000000095
:10BBB0000000000000000000000000000000000085
:10BBC0000000000000000004000100040001000764
:10BBD000FFFF000FFFFF000100C100020041000451
:10BBE00000200004002000040020000400200006C3
:10BBF0000040000301C00001FF8000007E00000043
:10BC00000000000000000000000000000000000034
:10BC10000000000000000000000000000000000024
:10BC20000000000000000000000000000000000014
:10BC30000000000000000000000000000000000004
:10BC40000000000000000000000000007E00000175
:10BC5000FF80000380C00002006000040020000498
:10BC60000020000400200004002000020041000326
:10BC700000C10003FFFF0007FFFF000000010000FC
:10BC800000010000000000000000000000000000B3
:10BC900000000000000000000000000000000000A4
:10BCA0000000000000000000000000000000000094
:10BCB0000000000000000000000000000000000084
:10BCC0000000000000000004002000040020000428
:10BCD000002000040020000FFFE0000FFFE0000044
:10BCE000C020000100200002002000060020000407
:10BCF0000000000400000007000000030000000036
:10BD00000000000000000000000000000000000033
:10BD10000000000000000000000000000000000023
:10BD20000000000000000000000000000000000013
:10BD30000000000000000000000000000000000003
:10BD400000000000000000000000000003E000010F
:10BD5000C0E00003E0400006302000043020000472
:10BD60001820000418200004182000040C200002F1
:10BD70000C60000307C00007838000000000000083
:10BD800000000000000000000000000000000000B3
:10BD900000000000000000000000000000000000A3
:10BDA0000000000000000000000000000000000093
:10BDB0000000000000000000000000000000000083
:10BDC000000000000000000000000004000000046B
:10BDD000000000040000000C0000001FFF8000FFB6
:10BDE000FFC00004006000040020000400200004E4
:10BDF000002000040040000001800000000000005E
:10BE00000000000000000000000000000000000032
:10BE10000000000000000000000000000000000022
:10BE20000000000000000000000000000000000012
:10BE30000000000000000000000000000000000002
:10BE400000000000000000040000000400000007E3
:10BE5000FF80000FFFC00000006000000020000015
:10BE6000002000000020000000200004004000042A
:10BE700000800007FFE0000FFFC00000004000004E
:10BE80000040000000000000000000000000000072
:10BE900000000000000000000000000000000000A2
:10BEA0000000000000000000000000000000000092
:10BEB0000000000000000000000000000000000082
:10BEC0000000000000000004000000040000000763
:10BED00080000007F0000004FE0000041FC0000006
:10BEE00003E00000038000001C0000046000000765
:10BEF00080000006000000040000000000000000B8
:10BF00000000000000000000000000000000000031
:10BF10000000000000000000000000000000000021
:10BF20000000000000000000000000000000000011
:10BF30000000000000000000000000000000000001
:10BF4000000000040000000600000007C000000719
:10BF5000FC0000043F80000003E000040F800006A6
:10BF6000F0000007F0000007FF8000040FE0000071
:10BF7000038000043C000007C0000006000000042D
:10BF800000000000000000000000000000000000B1
:10BF900000000000000000000000000000000000A1
:10BFA0000000000000000000000000000000000091
:10BFB0000000000000000000000000000000000081
:10BFC0000000000000000000002000040020000429
:10BFD0000060000700E0000783200007E60000047F
:10BFE000F80000003C0000045E20000587A0000669
:10BFF00001E00004006000040020000000200000B8
:10C000000000000000000000000000000000000030
:10C010000000000000000000000000000000000020
:10C020000000000000000000000000000000000010
:10C030000000000000000000000000000000000000
:10C0400000000000000000040000000400030007DE
:10C0500000030007E0010004F80100041F020000D3
:10C0600007FC000000E000000700000438000007A3
:10C07000C0000006000000040000000400000000F2
:10C0800000000000000000000000000000000000B0
:10C0900000000000000000000000000000000000A0
:10C0A0000000000000000000000000000000000090
:10C0B0000000000000000000000000000000000080
:10C0C0000000000000000000000000078060000683
:10C0D00000E0000403E0000407A000040E200004B8
:10C0E0003C20000470200005E020000780200007AD
:10C0F0000060000400E00000038000000000000079
:10C10000000000000000000000000000000000002F
:10C11000000000000000000000000000000000001F
:10C12000000000000000000000000000000000000F
:10C1300000000000000000000000000000000000FF
:10C1400000000000000000000000000000000000EF
:10C1500000000000000000000000000000000000DF
:10C160008000000080000001400007FE3FF808004A
:10C170000004100000021000000200000000000097
:10C1800000000000000000000000000000000000AF
:10C19000000000000000000000000000000000009F
:10C1A000000000000000000000000000000000008F
:10C1B000000000000000000000000000000000007F
:10C1C000000000000000000000000000000000006F
:10C1D000000000000000000000000000000000005F
:10C1E0000000FFFFFFFF0000000000000000000053
:10C1F000000000000000000000000000000000003F
:10C20000000000000000000000000000000000002E
:10C21000000000000000000000000000000000001E
:10C22000000000000000000000000000000000000E
:10C2300000000000000000000000000000000000FE
:10C2400000000000000000000000100000021000CC
:10C2500000020800000407FE3FF800014000000053
:10C2600080000000800000000000000000000000CE
:10C2700000000000000000000000000000000000BE
:10C2800000000000000000000000000000000000AE
:10C29000000000000000000000000000000000009E
:10C2A000000000000000000000000000000000008E
:10C2B000000000000000000000000000000000007E
:10C2C00000000000000018000000300000004000E6
:10C2D000000040000000400000002000000030008E
:10C2E000000008000000040000000200000002003E
:10C2F0000000020000000C00000018000000000018
:10C30000000000000000000000000000000000002D
:10C31000000000000000000000000000000000001D
:10C32000000000000000000000000000000000000D
:10C3300000000000000000000000000000000000FD
:10C34000000000000010000001000000000F0000CD
:10C35000C003000080070000C00300004000000090
:10C3600040000000400000004000000040000000CD
:10C3700040000000000004004000000000C0030076
:10C3800000F0000000E0010000F000003031323326
:10C3900034353637383941424344454640305800F9
:10C3A000303132333435363738396162636465662B
:10C3B00040307800D4C30008000000247C00000056
:10C3C000D402000850C400087C000024A4510400DA
:10C3D000F00200080090D0030090D003000000009D
:10C3E000000000000000000001000000100000003C
:10C3F0000000000001000000000000FFFFFFFFFF41
:10C40000000000000000000000000000000000002C
:10C410000D7A0008397A0008C005002400401FC0CA
:10C420000000003000000038000000200000000084
:10C43000C005042440401FC000C0033000F0003895
:10C4400000E0012000F000000000000000000000FB
:040000050800029954
:00000001FF
